:020000040000FA
:0408000044EF08F0C9
:1008100003B213EF05F0F2B431EF05F09EB039EFFB
:1008200005F09EB241EF05F0F2A81AEF04F0F2B223
:1008300025EF04F0F2A620EF04F0F2B022EF04F06E
:10084000F3EF07F0F296F290FF00CD90F2929EA0A7
:100850002FEF04F00101533F2FEF04F0542BAEC1F2
:10086000B2F1AFC1B3F1B0C1B4F1B1C1B5F1AAC138
:10087000AEF1ABC1AFF1ACC1B0F1ADC1B1F1A6C148
:10088000AAF1A7C1ABF1A8C1ACF1A9C1ADF1A2C158
:10089000A6F1A3C1A7F1A4C1A8F1A5C1A9F19EC168
:1008A000A2F19FC1A3F1A0C1A4F1A1C1A5F19AC178
:1008B0009EF19BC19FF19CC1A0F19DC1A1F196C188
:1008C0009AF197C19BF198C19CF199C19DF1CECF4E
:1008D00096F1CFCF97F153C198F154C199F1CF6AF6
:1008E000CE6A0101536B546B9E90CD800FBC0F8E6E
:1008F0000FBA7EEF04F00F8AF3EF07F00F8C0FBEF4
:10090000BAEF04F096C19AF197C19BF198C19CF19E
:1009100099C19DF19AC19EF19BC19FF19CC1A0F12B
:100920009DC1A1F19EC1A2F19FC1A3F1A0C1A4F1FB
:10093000A1C1A5F1A2C1A6F1A3C1A7F1A4C1A8F1CB
:10094000A5C1A9F1A6C1AAF1A7C1ABF1A8C1ACF19B
:10095000A9C1ADF1AAC1AEF1ABC1AFF1ACC1B0F16B
:10096000ADC1B1F1AEC1B2F1AFC1B3F1B0C1B4F13B
:10097000B1C1B5F101015E6B5F6B606B616B96514C
:100980005E2797515F2398516023995161239A51B3
:100990005E279B515F239C5160239D5161239E5193
:1009A0005E279F515F23A0516023A1516123A25173
:1009B0005E27A3515F23A4516023A5516123A65153
:1009C0005E27A7515F23A8516023A9516123AA5133
:1009D0005E27AB515F23AC516023AD516123AE5113
:1009E0005E27AF515F23B0516023B1516123B251F3
:1009F0005E27B3515F23B4516023B5516123D89072
:100A00000101613360335F335E33D890010161339C
:100A100060335F335E33D8900101613360335F33FD
:100A20005E33F3EF07F00392ABB2AB98AB880301F0
:100A300003EE00F080517F0BE92604C0EFFF802B0E
:100A40008151805D700BD8A48B8200008051815D44
:100A5000700BD8A48B9281518019D8B40790F3EF12
:100A600007F0F2940101453FF3EF07F0462BF3EF57
:100A700007F09E900101533FF3EF07F0542BF3EF83
:100A800007F09E92040062A146EF05F007B498EFCC
:100A900005F007B098EF05F01EC620F61FC621F638
:100AA0001CC61EF61DC61FF61AC61CF61BC61DF672
:100AB00006C608F607C609F604C606F605C607F612
:100AC00002C604F603C605F626C628F627C629F68A
:100AD00024C626F625C627F622C624F623C625F602
:100AE0000EC610F60FC611F60CC60EF60DC60FF6A2
:100AF0000AC60CF60BC60DF62EC630F62FC631F61A
:100B00002CC62EF62DC62FF62AC62CF62BC62DF691
:100B100016C618F617C619F614C616F615C617F631
:100B200012C614F613C615F608EC2CF0A0EC2BF048
:100B3000077C07ACB3EF05F0C274C2B4ADEF05F0AB
:100B4000C3CFB3F5C4CFB4F50501D890B433B333F4
:100B5000D890B433B333B4EF05F0C3CF55F1C4CF5D
:100B600056F1B4EF05F0C28207B421EF06F047C199
:100B70004BF148C14CF149C14DF14AC14EF15EC142
:100B800062F15FC163F160C164F161C165F196C159
:100B9000B6F197C1B7F198C1B8F199C1B9F19AC14D
:100BA000BAF19BC1BBF19CC1BCF19DC1BDF19EC11D
:100BB000BEF19FC1BFF1A0C1C0F1A1C1C1F1A2C1ED
:100BC000C2F1A3C1C3F1A4C1C4F1A5C1C5F1A6C1BD
:100BD000C6F1A7C1C7F1A8C1C8F1A9C1C9F1AAC18D
:100BE000CAF1ABC1CBF1ACC1CCF1ADC1CDF1AEC15D
:100BF000CEF1AFC1CFF1B0C1D0F1B1C1D1F1B2C12D
:100C0000D2F1B3C1D3F1B4C1D4F1B5C1D5F1B3C5FB
:100C1000B5F5B4C5B6F5B5C5B7F5B6C5B8F50101B6
:100C200055515B2756515C23E86A5D230E2E21EF58
:100C300006F05CC157F15DC158F15B6B5C6B5D6B9D
:100C4000078E0201002FF3EF07F03C0E006F00C18A
:100C50000CF101C10DF102C10EF103C10FF104C18C
:100C600010F105C111F106C112F107C113F108C15C
:100C700014F109C115F10AC116F10BC117F134C104
:100C800035F105012F51000AD8B4F2EF06F0050145
:100C90002F51010AD8B47CEF06F005012F51020A4A
:100CA000D8B4BDEF06F005012F51030AD8B4BDEF4B
:100CB00006F005012F51040AD8B4BDEF06F0050176
:100CC0002F51050AD8B4BDEF06F005012F51060AD1
:100CD000D8B4BDEF06F005012F51070AD8B4BDEF17
:100CE00006F005012F51320AD8B47AEF06F02F6BC7
:100CF000F2EF06F0F2EF06F00501536787EF06F01A
:100D0000546787EF06F0556787EF06F056678BEF5D
:100D100006F0F2EF06F057C500F158C501F159C5CC
:100D200002F15AC503F10101010E046F000E056FB7
:100D3000000E066F000E076F11EC2AF000C157F588
:100D400001C158F502C159F503C15AF50067B0EF6A
:100D500006F00167B0EF06F00267B0EF06F0036738
:100D6000F2EF06F053C557F554C558F555C559F57A
:100D700056C55AF50F88F2EF06F005013067C3EF4C
:100D800006F0F2EF06F00FBED8EF06F010A0DDEF90
:100D900006F001014767D4EF06F04867D4EF06F08C
:100DA0004967D4EF06F04A67D8EF06F0DDEF06F0AA
:100DB00007AEDDEF06F0EFEF06F00501312FF2EFA1
:100DC00006F03C0E316F302FF2EF06F00101000EFD
:100DD000626FE00E636FA50E646F010E656F050113
:100DE000306B0F880501626B33B7F8EF06F0628154
:100DF0000CC100F10DC101F10EC102F10FC103F1EF
:100E000010C104F111C105F112C106F113C107F1BE
:100E100014C108F115C109F116C10AF117C10BF18E
:100E200035C134F100C10CF101C10DF102C10EF167
:100E300003C10FF104C110F105C111F106C112F196
:100E400007C113F108C114F109C115F10AC116F166
:100E50000BC117F134C135F101018A6737EF07F093
:100E60008B6737EF07F08C6737EF07F08D673BEF45
:100E700007F06BEF07F08EC100F18FC101F190C157
:100E800002F191C103F10101010E046F000E056F23
:100E9000000E066F000E076F11EC2AF000C18EF1F4
:100EA00001C18FF102C190F103C191F1006760EFC0
:100EB00007F0016760EF07F0026760EF07F0036774
:100EC0006BEF07F08AC18EF18BC18FF18CC190F16D
:100ED0008DC191F10F80D57ED5BE69D0D6CF47F1B7
:100EE000D7CF48F145C149F1E86AE8CF4AF11090FF
:100EF00047C100F148C101F149C102F14AC103F102
:100F000001010A0E046F000E056F000E066F000E41
:100F1000076F11EC2AF003AF1080010154A79DEF79
:100F200007F00F9A0F9C0F9E0101000E5E6F600E7E
:100F30005F6F3D0E606F080E616F010147BFADEF3F
:100F400007F04867ADEF07F04967ADEF07F04A6774
:100F5000ADEF07F0F288D2EF07F0F2985E6B5F6BAF
:100F6000606B616B966B976B986B996B9A6B9B6BD5
:100F70009C6B9D6B9E6B9F6BA06BA16BA26BA36B1D
:100F8000A46BA56BA66BA76BA86BA96BAA6BAB6BCD
:100F9000AC6BAD6BAE6BAF6BB06BB16BB26BB36B7D
:100FA000B46BB56BD76AD66A0101456B466B0CC151
:100FB00000F10DC101F10EC102F10FC103F110C129
:100FC00004F111C105F112C106F113C107F114C1F9
:100FD00008F115C109F116C10AF117C10BF135C1AC
:100FE00034F1F3EF07F002C0E0FF005001C0D8FF7A
:100FF0001000A6B2F9EF07F00CC0A9FF0BC0A8FFC4
:10100000A69EA69CA684F29E550EA76EAA0EA76E5B
:10101000A682F28EA694A6B20BEF08F00C2A12005C
:10102000A96EA69EA69CA680A8500C2A12000401B8
:101030002C0E826F3EEC0BF00CEC2BF00C5010ECF5
:1010400008F0E8CF00F10C5010EC08F0E8CF01F107
:1010500001AF30EF08F00101FF0E026FFF0E036FCA
:10106000AFEC2AF029673CEF08F00401200E826FF4
:101070003EEC0BF041EF08F004012D0E826F3EECC8
:101080000BF0D9EC28F01200076A0F6A106A0F0102
:101090000D0EC16E860EC06E030EC26E0F01680E7D
:1010A000896E130E926E080E8A6E8A6AF30E936E24
:1010B0008B6A900E946EF18EF19E0E6A01015B6B4D
:1010C0005C6B5D6B576B586BF29A0101476B486B19
:1010D000496B4A6B4B6B4C6B4D6B4E6B4F6B506B54
:1010E000516B526B456B466BD76AD66A0F01280E5F
:1010F000D56EF28A9D90B00ECD6E01015E6B5F6B76
:10110000606B616B626B636B646B656B666B676B6B
:10111000686B696B536B546BCF6ACE6A0F9A0F9CE6
:101120000F9E9D80760ECA6E9D8202013C0E006F5E
:10113000CC6A160E10EC08F0E8CF00F1170E10EC98
:1011400008F0E8CF01F1180E10EC08F0E8CF02F13A
:10115000190E10EC08F0E8CF03F1010103AFCBEF5B
:1011600008F00CEC2BF0160E0C6E00C10BF0F9EC35
:1011700007F0170E0C6E01C10BF0F9EC07F0180E1A
:101180000C6E02C10BF0F9EC07F0190E0C6E03C1E6
:101190000BF0F9EC07F000C18AF101C18BF102C13B
:1011A0008CF103C18DF100C18EF101C18FF102C13B
:1011B00090F103C191F11A0E10EC08F0E8CF00F1A4
:1011C0001B0E10EC08F0E8CF01F11C0E10EC08F03B
:1011D000E8CF02F11D0E10EC08F0E8CF03F1010199
:1011E00003AF21EF09F00CEC2BF01A0E0C6E00C1CE
:1011F0000BF0F9EC07F01B0E0C6E01C10BF0F9ECD3
:1012000007F01C0E0C6E02C10BF0F9EC07F01D0E7E
:101210000C6E03C10BF0F9EC07F01A0E10EC08F09D
:10122000E8CF00F11B0E10EC08F0E8CF01F11C0E26
:1012300010EC08F0E8CF02F11D0E10EC08F0E8CF3A
:1012400003F100C192F101C193F102C194F103C114
:1012500095F1240EAC6E900EAB6E240EAC6E080EA3
:10126000B86E000EB06E1F0EAF6E0401806B816B06
:101270000F01900EAB6E0F019D8A0301806B816B95
:10128000C26B8B929DEC31F09DEC31F0880E10EC2E
:1012900008F0E8CF00F1890E10EC08F0E8CF01F17A
:1012A000010101AF6CEF09F00CEC2BF0880E0C6E15
:1012B00000C10BF0F9EC07F0890E0C6E01C10BF0C8
:1012C000F9EC07F0880E10EC08F0E8CF00F1890E79
:1012D00010EC08F0E8CF01F100C140F601C141F681
:1012E00002C142F603C143F6F5EC34F07CEC2FF07A
:1012F000200E10EC08F0E8CF2FF505012F51FF0A62
:10130000D8A48AEF09F02F6B200E0C6E2FC50BF0BE
:10131000F9EC07F00501010E306F3C0E316F250E20
:1013200010EC08F0E8CF00F1260E10EC08F0E8CF42
:1013300001F1270E10EC08F0E8CF02F1280E10ECB6
:1013400008F0E8CF03F1010103AFC1EF09F00CECA5
:101350002BF0250E0C6E00C10BF0F9EC07F0260EF9
:101360000C6E01C10BF0F9EC07F0270E0C6E02C1F8
:101370000BF0F9EC07F0280E0C6E03C10BF0F9EC42
:1013800007F000C153F501C154F502C155F503C181
:1013900056F500C157F501C158F502C159F503C111
:1013A0005AF5290E10EC08F0E8CF5BF505015C5109
:1013B0005B5DD8A05BC55CF505012F51020A0EE10B
:1013C00081B8EEEF09F005015C2FEBEF09F05BC58A
:1013D0005CF5EEEF09F081BA34EF35F0210E10EC38
:1013E00008F0E8CF00F1220E10EC08F0E8CF01F190
:1013F000230E10EC08F0E8CF02F1240E10EC08F0F8
:10140000E8CF03F1010103AF34EF0AF00CEC2BF04D
:10141000210E0C6E00C10BF0F9EC07F0220E0C6EE1
:1014200001C10BF0F9EC07F0230E0C6E02C10BF0BA
:10143000F9EC07F0240E0C6E03C10BF0F9EC07F089
:10144000210E10EC08F0E8CF00F1220E10EC08F0AD
:10145000E8CF01F1230E10EC08F0E8CF02F1240EE2
:1014600010EC08F0E8CF03F100C15DF501C15EF5B5
:1014700002C15FF503C160F5B3EC2EF075EC2DF001
:10148000C5EC2CF005012F51030A12E005012F5184
:10149000040A1DE005012F51050A24E005012F5122
:1014A000060A32E005012F51070A38E097EF0AF0EB
:1014B000ACC500F101010F0E001701010051000A37
:1014C00036E001010051050A32E094EF0AF0ACC5A4
:1014D00000F101010F0E001701010051000A27E081
:1014E00094EF0AF00501AC51000A21E00501AC516E
:1014F000150A1DE00501AC51300A19E00501AC5197
:10150000450A15E094EF0AF00501AC51000A0FE01E
:101510000501AC51300A0BE094EF0AF00501AC5123
:10152000000A05E094EF0AF081BA34EF35F070EC70
:101530002CF007900001F28EF28C07B06DEF26F0D0
:101540000FB04CEF21F00FB810EF1BF003018051EA
:1015500081197F0BD8B46DEF26F013EE00F08151A6
:101560007F0BE126812BE7CFE8FFE00BD8B46DEFCE
:1015700026F023EE82F0C2513F0BD926E7CFDFFFE2
:10158000C22BDF50780AD8A46DEF26F007808EC1F9
:1015900000F18FC101F190C102F191C103F101018C
:1015A000040E046F000E056F000E066F000E076F2D
:1015B00011EC2AF000AFE6EF0AF00101030E8E6F86
:1015C000000E8F6F000E906F000E916F030182511D
:1015D000720AD8B44CEF21F08251520AD8B44CEFC1
:1015E00021F08251750AD8B44CEF21F08251630A80
:1015F000D8B427EF23F08251690AD8B407EF1EF060
:1016000082517A0AD8B41AEF1FF08251490AD8B42D
:10161000A6EF1DF08251500AD8B4C4EF1CF08251DD
:10162000700AD8B407EF1DF08251540AD8B432EFD3
:101630001DF08251740AD8B478EF1DF082516D0A02
:10164000D8B452EF0BF082514D0AD8B46BEF0BF0C7
:101650008251730AD8B47CEF20F08251530AD8B477
:10166000E1EF20F082514C0AD8B4CEEF12F0825153
:10167000760AD8B4FAEF0BF05EEF23F0040114EE13
:1016800000F080517F0BE12682C4E7FF802B12001F
:1016900004010D0E826F3EEC0BF00A0E826F3EECE1
:1016A0000BF0120004016D0E826F3EEC0BF0030193
:1016B0008351300AD8B4AAEF0BF003018351310AE9
:1016C000D8B4BDEF0BF003018351320AD8B4D0EF88
:1016D0000BF05EEF23F004014D0E826F3EEC0BF039
:1016E0004DEC2BF084C331F185C332F186C333F165
:1016F0000101296B5AEC2BF0D1EC2AF00301835144
:10170000300AD8B492EF0BF003018351310AD8B4F8
:101710009AEF0BF003018351320AD8B4A2EF0BF019
:101720005EEF23F0FD0E0C6E00C10BF0F9EC07F03C
:10173000AAEF0BF0FE0E0C6E00C10BF0F9EC07F0F7
:10174000BDEF0BF0FF0E0C6E00C10BF0F9EC07F0D3
:10175000D0EF0BF00401300E826F3EEC0BF0040171
:101760002C0E826F3EEC0BF00CEC2BF0FD0E10EC0F
:1017700008F0E8CF00F1E1EF0BF00401310E826FC9
:101780003EEC0BF004012C0E826F3EEC0BF00CECE7
:101790002BF0FE0E10EC08F0E8CF00F1E1EF0BF0BB
:1017A0000401320E826F3EEC0BF00CEC2BF00401C6
:1017B0002C0E826F3EEC0BF0FF0E10EC08F0E8CF21
:1017C00000F1AFEC2AF031C182F40401300E82271F
:1017D0003EEC0BF032C182F40401300E82273EEC65
:1017E0000BF033C182F40401300E82273EEC0BF083
:1017F0005CEF23F003018351300AD8B49FEF0DF062
:1018000003018351310AD8B4D6EF0DF0030183519F
:10181000320AD8B48BEF0FF003018351330AD8B4E6
:1018200040EF11F003018351340AD8B4E6EF11F010
:1018300003018351730AD8B481EF0CF00301835183
:10184000760AD8B483EF0CF003018351740AD8B43C
:101850006EEF0CF003018351540AD8B433EF0CF04F
:10186000D8A45EEF23F00401760E826F3EEC0BF0FD
:101870000401540E826F3EEC0BF007840001880EC9
:101880000C6E4DEC2BF02981030184512D0AD8B444
:101890004CEF0CF00101299185C32FF186C330F183
:1018A00087C331F188C332F189C333F15AEC2BF08D
:1018B000D1EC2AF000C10BF0F9EC07F001C10BF0FC
:1018C000F9EC07F0880E10EC08F0E8CF40F6890E2E
:1018D00010EC08F0E8CF41F679EF0CF00401760E39
:1018E000826F3EEC0BF00401740E826F3EEC0BF045
:1018F00007840001880E0C6E17EC08F0079471EF56
:101900001BF081EC0CF00401760E826F3EEC0BF0C4
:101910000401760E826F3EEC0BF0078489EC27F011
:1019200004012C0E826F3EEC0BF00101036B026B85
:101930003BC601F13AC600F101AFA4EF0CF0010182
:10194000FF0E026FFF0E036FAFEC2AF02967ABEFBB
:101950000CF0B0EF0CF004012D0E826F3EEC0BF09A
:101960002FC182F40401300E82273EEC0BF030C10F
:1019700082F40401300E82273EEC0BF031C182F478
:101980000401300E82273EEC0BF032C182F40401D8
:10199000300E82273EEC0BF033C182F40401300E8E
:1019A00082273EEC0BF004012C0E826F3EEC0BF014
:1019B0000101036B026B3DC601F13CC600F101AFB2
:1019C000E7EF0CF00101FF0E026FFF0E036FAFECAB
:1019D0002AF02967EEEF0CF0F3EF0CF004012D0E66
:1019E000826F3EEC0BF02FC182F40401300E82278F
:1019F0003EEC0BF030C182F40401300E82273EEC45
:101A00000BF031C182F40401300E82273EEC0BF062
:101A100032C182F40401300E82273EEC0BF033C158
:101A200082F40401300E82273EEC0BF004012C0EF0
:101A3000826F3EEC0BF00101036B026B3FC601F1BC
:101A40003EC600F101AF2AEF0DF00101FF0E026F5B
:101A5000FF0E036FAFEC2AF0296731EF0DF036EF80
:101A60000DF004012D0E826F3EEC0BF02FC182F4BD
:101A70000401300E82273EEC0BF030C182F40401E9
:101A8000300E82273EEC0BF031C182F40401300E9F
:101A900082273EEC0BF032C182F40401300E822723
:101AA0003EEC0BF033C182F40401300E82273EEC91
:101AB0000BF004012C0E826F3EEC0BF00101036B66
:101AC000026B37C601F136C600F101AF6DEF0DF0C4
:101AD0000101FF0E026FFF0E036FAFEC2AF02967C2
:101AE00074EF0DF079EF0DF004012D0E826F3EECD6
:101AF0000BF02FC182F40401300E82273EEC0BF074
:101B000030C182F40401300E82273EEC0BF031C16B
:101B100082F40401300E82273EEC0BF032C182F4D5
:101B20000401300E82273EEC0BF033C182F4040135
:101B3000300E82273EEC0BF0079471EF1BF004018E
:101B4000760E826F3EEC0BF00401300E826F3EEC9D
:101B50000BF004012C0E826F3EEC0BF07AEC2BF0B4
:101B60000CEC2BF000C600F101C601F1AFEC2AF03D
:101B700030C182F40401300E82273EEC0BF031C1FB
:101B800082F40401300E82273EEC0BF032C182F465
:101B90000401300E82273EEC0BF033C182F40401C5
:101BA000300E82273EEC0BF071EF1BF00401760E35
:101BB000826F3EEC0BF00401310E826F3EEC0BF0B5
:101BC00007840101036B026B02C600F103C601F139
:101BD00001AFEFEF0DF0FF0E026FFF0E036F01017B
:101BE000076B066B04C604F105C605F105AFFDEFF2
:101BF0000DF0FF0E066FFF0E076F16EC2AF00101C5
:101C0000076B066B06C604F107C605F105AF0DEFBD
:101C10000EF0FF0E066FFF0E076F16EC2AF00101A3
:101C2000076B066B08C604F109C605F105AF1DEF89
:101C30000EF0FF0E066FFF0E076F16EC2AF0D8901D
:101C400001010333023301330033D8900101033320
:101C500002330133003304012C0E826F3EEC0BF093
:101C60000101036B026B01C101F100C100F101AF81
:101C70003FEF0EF00101FF0E026FFF0E036FAFEC9E
:101C80002AF0296746EF0EF04BEF0EF004012D0EFF
:101C9000826F3EEC0BF02FC182F40401300E8227DC
:101CA0003EEC0BF030C182F40401300E82273EEC92
:101CB0000BF031C182F40401300E82273EEC0BF0B0
:101CC00032C182F40401300E82273EEC0BF033C1A6
:101CD00082F40401300E82273EEC0BF00101036B0D
:101CE000026B0AC600F10BC601F101AF7CEF0EF0EA
:101CF000FF0E026FFF0E036F0101076B066B0CC630
:101D000004F10DC605F105AF8AEF0EF0FF0E066F68
:101D1000FF0E076F16EC2AF00101076B066B0EC66B
:101D200004F10FC605F105AF9AEF0EF0FF0E066F36
:101D3000FF0E076F16EC2AF00101076B066B10C649
:101D400004F111C605F105AFAAEF0EF0FF0E066F04
:101D5000FF0E076F16EC2AF0D8900101033302330F
:101D600001330033D89001010333023301330033D0
:101D700004012C0E826F3EEC0BF00101036B026B31
:101D800001C101F100C100F101AFCCEF0EF0010182
:101D9000FF0E026FFF0E036FAFEC2AF02967D3EF3F
:101DA0000EF0D8EF0EF004012D0E826F3EEC0BF01A
:101DB0002FC182F40401300E82273EEC0BF030C1BB
:101DC00082F40401300E82273EEC0BF031C182F424
:101DD0000401300E82273EEC0BF032C182F4040184
:101DE000300E82273EEC0BF033C182F40401300E3A
:101DF00082273EEC0BF00101036B026B12C600F16F
:101E000013C601F101AF09EF0FF0FF0E026FFF0ED5
:101E1000036F0101076B066B14C604F115C605F1CB
:101E200005AF17EF0FF0FF0E066FFF0E076F16ECF2
:101E30002AF00101076B066B16C604F117C605F1FF
:101E400005AF27EF0FF0FF0E066FFF0E076F16ECC2
:101E50002AF00101076B066B18C604F119C605F1DB
:101E600005AF37EF0FF0FF0E066FFF0E076F16EC92
:101E70002AF0D89001010333023301330033D890A4
:101E80000101033302330133003304012C0E826F4E
:101E90003EEC0BF00101036B026B01C101F100C1CB
:101EA00000F101AF59EF0FF00101FF0E026FFF0EBD
:101EB000036FAFEC2AF0296760EF0FF065EF0FF0CA
:101EC00004012D0E826F3EEC0BF02FC182F4040151
:101ED000300E82273EEC0BF030C182F40401300E4C
:101EE00082273EEC0BF031C182F40401300E8227D0
:101EF0003EEC0BF032C182F40401300E82273EEC3E
:101F00000BF033C182F40401300E82273EEC0BF05B
:101F1000079471EF1BF00401760E826F3EEC0BF01C
:101F20000401320E826F3EEC0BF007840101036B5B
:101F3000026B1AC600F11BC601F101AFA4EF0FF04E
:101F4000FF0E026FFF0E036F0101076B066B1CC6CD
:101F500004F11DC605F105AFB2EF0FF0FF0E066FDD
:101F6000FF0E076F16EC2AF00101076B066B1EC609
:101F700004F11FC605F105AFC2EF0FF0FF0E066FAB
:101F8000FF0E076F16EC2AF00101076B066B20C6E7
:101F900004F121C605F105AFD2EF0FF0FF0E066F79
:101FA000FF0E076F16EC2AF0D890010103330233BD
:101FB00001330033D890010103330233013300337E
:101FC00004012C0E826F3EEC0BF00101036B026BDF
:101FD00001C101F100C100F101AFF4EF0FF0010107
:101FE000FF0E026FFF0E036FAFEC2AF02967FBEFC5
:101FF0000FF000EF10F004012D0E826F3EEC0BF09D
:102000002FC182F40401300E82273EEC0BF030C168
:1020100082F40401300E82273EEC0BF031C182F4D1
:102020000401300E82273EEC0BF032C182F4040131
:10203000300E82273EEC0BF033C182F40401300EE7
:1020400082273EEC0BF00101036B026B22C600F10C
:1020500023C601F101AF31EF10F0FF0E026FFF0E4A
:10206000036F0101076B066B24C604F125C605F159
:1020700005AF3FEF10F0FF0E066FFF0E076F16EC77
:102080002AF00101076B066B26C604F127C605F18D
:1020900005AF4FEF10F0FF0E066FFF0E076F16EC47
:1020A0002AF00101076B066B28C604F129C605F169
:1020B00005AF5FEF10F0FF0E066FFF0E076F16EC17
:1020C0002AF0D89001010333023301330033D89052
:1020D0000101033302330133003304012C0E826FFC
:1020E0003EEC0BF00101036B026B01C101F100C179
:1020F00000F101AF81EF10F00101FF0E026FFF0E42
:10210000036FAFEC2AF0296788EF10F08DEF10F025
:1021100004012D0E826F3EEC0BF02FC182F40401FE
:10212000300E82273EEC0BF030C182F40401300EF9
:1021300082273EEC0BF031C182F40401300E82277D
:102140003EEC0BF032C182F40401300E82273EECEB
:102150000BF033C182F40401300E82273EEC0BF009
:102160000101036B026B2AC600F12BC601F101AF1E
:10217000BEEF10F0FF0E026FFF0E036F0101076B41
:10218000066B2CC604F12DC605F105AFCCEF10F09F
:10219000FF0E066FFF0E076F16EC2AF00101076BAA
:1021A000066B2EC604F12FC605F105AFDCEF10F06B
:1021B000FF0E066FFF0E076F16EC2AF00101076B8A
:1021C000066B30C604F131C605F105AFECEF10F037
:1021D000FF0E066FFF0E076F16EC2AF0D890010174
:1021E0000333023301330033D89001010333023348
:1021F0000133003304012C0E826F3EEC0BF0010121
:10220000036B026B01C101F100C100F101AF0EEFE0
:1022100011F00101FF0E026FFF0E036FAFEC2AF009
:10222000296715EF11F01AEF11F004012D0E826FDE
:102230003EEC0BF02FC182F40401300E82273EECFD
:102240000BF030C182F40401300E82273EEC0BF01B
:1022500031C182F40401300E82273EEC0BF032C112
:1022600082F40401300E82273EEC0BF033C182F47D
:102270000401300E82273EEC0BF0079471EF1BF047
:102280000401760E826F3EEC0BF00401330E826F78
:102290003EEC0BF004012C0E826F3EEC0BF085C37C
:1022A00082F43EEC0BF0640E0D6E03018551320A90
:1022B00002E16A0E0D6E03018551330A02E1700ED0
:1022C0000D6E03018551340A02E1760E0D6E030195
:1022D0008551350A02E17C0E0D6E03018551360AE7
:1022E00002E1820E0D6E03018651780A65E00DC091
:1022F0000CF04DEC2BF02981030187512D0AD8B445
:1023000084EF11F00101299188C32FF189C330F1C5
:102310008AC331F18BC332F18CC333F15AEC2BF009
:10232000D1EC2AF000C10BF0F9EC07F001C10BF081
:10233000F9EC07F04DEC2BF0298103018E512D0AA9
:10234000D8B4A5EF11F0010129918FC32FF190C3EB
:1023500030F191C331F192C332F193C333F15AECAE
:102360002BF0D1EC2AF000C10BF0F9EC07F001C121
:102370000BF0F9EC07F04DEC2BF02981030195519E
:102380002D0AD8B4C6EF11F00101299196C32FF19F
:1023900097C330F198C331F199C332F19AC333F145
:1023A0005AEC2BF0D1EC2AF000C10BF0F9EC07F05D
:1023B00001C10BF0F9EC07F00DC00CF017EC08F0C0
:1023C00017EC08F017EC08F071EF1BF00401760E23
:1023D000826F3EEC0BF00401340E826F3EEC0BF08A
:1023E00003018451780AD8B4BEEF12F03E0E0C6E91
:1023F0004DEC2BF02981030185512D0AD8B403EF50
:1024000012F00101299186C32FF187C330F188C3EF
:1024100031F189C332F18AC333F15AEC2BF0D1EC9C
:102420002AF000C10BF0F9EC07F001C10BF0F9EC58
:1024300007F04DEC2BF0298103018C512D0AD8B403
:1024400024EF12F0010129918DC32FF18EC330F1D9
:102450008FC331F190C332F191C333F15AEC2BF0B9
:10246000D1EC2AF000C10BF0F9EC07F001C10BF040
:10247000F9EC07F04DEC2BF02981030193512D0A63
:10248000D8B445EF12F00101299194C32FF195C3FF
:1024900030F196C331F197C332F198C333F15AEC5E
:1024A0002BF0D1EC2AF000C10BF0F9EC07F001C1E0
:1024B0000BF0F9EC07F04DEC2BF0298103019A5158
:1024C0002D0AD8B466EF12F0010129919BC32FF1B8
:1024D0009CC330F19DC331F19EC332F19FC333F1F0
:1024E0005AEC2BF0D1EC2AF000C10BF0F9EC07F01C
:1024F00001C10BF0F9EC07F04DEC2BF02981030141
:10250000A1512D0AD8B487EF12F001012991A2C37D
:102510002FF1A3C330F1A4C331F1A5C332F1A6C397
:1025200033F15AEC2BF0D1EC2AF000C10BF0F9ECAE
:1025300007F001C10BF0F9EC07F04DEC2BF029810D
:102540000301A8512D0AD8B4A8EF12F00101299176
:10255000A9C32FF1AAC330F1ABC331F1ACC332F13F
:10256000ADC333F15AEC2BF0D1EC2AF000C10BF0E3
:10257000F9EC07F001C10BF0F9EC07F03E0E0C6E20
:1025800017EC08F017EC08F017EC08F017EC08F05F
:1025900017EC08F017EC08F071EF1BF00301835102
:1025A000300AD8B433EF16F003018351310AD8B49E
:1025B00041EF17F003018351320AD8B4AFEF17F09F
:1025C00003018351330AD8B4BFEF17F003018351DD
:1025D000340AD8B4CFEF17F003018351350AD8B4C9
:1025E00015EF1BF003018351360AD8B443EF1BF0FB
:1025F00003018351370AD8B495EF15F003018351D5
:10260000460AD8B469EF1AF0030183514D0AD8B4D1
:102610000EEF14F0030183516D0AD8B428EF14F0C3
:10262000030183515A0AD8B4BBEF16F0030183515A
:10263000490AD8B443EF1CF003018351500AD8B4BF
:1026400075EF1BF003018351540AD8B4EEEF1BF071
:1026500003018351630AD8B448EF14F00301835196
:10266000430AD8B440EF15F003018351730AD8B47C
:1026700046EF14F003018351610AD8B45BEF13F005
:1026800003018351650AD8B483EF16F00301835127
:10269000450AD8B491EF16F003018351620AD8B409
:1026A0009FEF16F003018351420AD8B4ADEF16F044
:1026B000D8A45EEF23F004014C0E826F3EEC0BF0C9
:1026C0000401610E826F3EEC0BF075EC2DF00401FD
:1026D0002C0E826F3EEC0BF00CEC2BF0ABC500F136
:1026E0000101AFEC2AF031C182F40401300E8227DF
:1026F0003EEC0BF032C182F40401300E82273EEC36
:102700000BF033C182F40401300E82273EEC0BF053
:1027100004012C0E826F3EEC0BF00CEC2BF0ACC5E0
:1027200000F10101AFEC2AF031C182F40401300E56
:1027300082273EEC0BF032C182F40401300E822776
:102740003EEC0BF033C182F40401300E82273EECE4
:102750000BF004012C0E826F3EEC0BF00CEC2BF016
:10276000ADC500F10101AFEC2AF031C182F40401E2
:10277000300E82273EEC0BF032C182F40401300EA1
:1027800082273EEC0BF033C182F40401300E822725
:102790003EEC0BF004012C0E826F3EEC0BF00CECC7
:1027A0002BF0AEC500F10101AFEC2AF031C182F48B
:1027B0000401300E82273EEC0BF032C182F404019A
:1027C000300E82273EEC0BF033C182F40401300E50
:1027D00082273EEC0BF004012C0E826F3EEC0BF0D6
:1027E0000CEC2BF0B3C500F10101AFEC2AF031C1C4
:1027F00082F40401300E82273EEC0BF032C182F4E9
:102800000401300E82273EEC0BF033C182F4040148
:10281000300E82273EEC0BF071EF1BF04DEC2BF0ED
:1028200084C333F15AEC2BF0D1EC2AF0200E0C6E5D
:1028300000C10BF0F9EC07F000C12FF505012F5195
:10284000000A06E005012F51010A02E01BEC2EF000
:1028500004014C0E826F3EEC0BF004014D0E826FB2
:102860003EEC0BF004012C0E826F3EEC0BF00CECF6
:102870002BF02FC500F1AFEC2AF033C182F4040134
:10288000300E82273EEC0BF071EF1BF034EF35F089
:1028900004014C0E826F3EEC0BF00401630E826F5C
:1028A0003EEC0BF0C5EC2CF004012C0E826F3EECDC
:1028B0000BF05DEC14F071EF1BF00CEC2BF0B1C5DC
:1028C00000F10101003B0F0E0017AFEC2AF033C1FD
:1028D00082F40401300E82273EEC0BF0B1C500F10A
:1028E00001010F0E01010017AFEC2AF033C182F491
:1028F0000401300E82273EEC0BF004012D0E826F96
:102900003EEC0BF0B0C500F10101003B0F0E0017CB
:10291000AFEC2AF033C182F40401300E82273EEC82
:102920000BF0B0C500F101010F0E01010017AFEC73
:102930002AF033C182F40401300E82273EEC0BF002
:1029400004012D0E826F3EEC0BF0AFC500F10101CA
:10295000003B0F0E0017AFEC2AF033C182F40401E4
:10296000300E82273EEC0BF0AFC500F101010F0ED7
:1029700001010017AFEC2AF033C182F40401300EDC
:1029800082273EEC0BF00401200E826F3EEC0BF030
:10299000AEC500F10F0E01010017AFEC2AF033C1F4
:1029A00082F40401300E82273EEC0BF00401200E6D
:1029B000826F3EEC0BF0ADC500F101010101003B5F
:1029C0000F0E0017AFEC2AF033C182F40401300E71
:1029D00082273EEC0BF0ADC500F101010F0E0101A5
:1029E0000017AFEC2AF033C182F40401300E8227C5
:1029F0003EEC0BF004013A0E826F3EEC0BF0ACC5DE
:102A000000F10101003B0F0E0017AFEC2AF033C1BB
:102A100082F40401300E82273EEC0BF0ACC500F1CD
:102A200001010F0E01010017AFEC2AF033C182F44F
:102A30000401300E82273EEC0BF004013A0E826F47
:102A40003EEC0BF0ABC500F10101003B0F0E00178F
:102A5000AFEC2AF033C182F40401300E82273EEC41
:102A60000BF0ABC500F101010F0E0017AFEC2AF01F
:102A700033C182F40401300E82273EEC0BF01200C9
:102A800084C3E8FF0F0BE83AE8CFB1F585C3E8FF50
:102A90000F0B0501B11387C3E8FF0F0BE83AE8CF2E
:102AA000B0F588C3E8FF0F0B0501B0138AC3E8FF38
:102AB0000F0BE83AE8CFAFF58BC3E8FF0F0B05012A
:102AC000AF138DC3E8FF0F0BE8CFAEF58FC3E8FF60
:102AD0000F0BE83AE8CFADF590C3E8FF0F0B050107
:102AE000AD1392C3E8FF0F0BE83AE8CFACF593C300
:102AF000E8FF0F0B0501AC1395C3E8FF0F0BE83A95
:102B0000E8CFABF596C3E8FF0F0B0501AB1324EC40
:102B10002DF004014C0E826F3EEC0BF00401430ECD
:102B2000826F3EEC0BF052EF14F0078404014C0E60
:102B3000826F3EEC0BF00401370E826F3EEC0BF01F
:102B400004012C0E826F3EEC0BF005012E51130A8E
:102B500006E005012E51170A0DE030EF16F00101D5
:102B6000000E006F000E016F100E026F000E036F5B
:102B7000C3EF15F00101000E006F000E016F000E93
:102B8000026F010E036FAFEC2AF02AC182F4040138
:102B9000300E82273EEC0BF02BC182F40401300E84
:102BA00082273EEC0BF02CC182F40401300E822708
:102BB0003EEC0BF02DC182F40401300E82273EEC76
:102BC0000BF02EC182F40401300E82273EEC0BF094
:102BD0002FC182F40401300E82273EEC0BF030C18D
:102BE00082F40401300E82273EEC0BF031C182F4F6
:102BF0000401300E82273EEC0BF032C182F4040156
:102C0000300E82273EEC0BF033C182F40401300E0B
:102C100082273EEC0BF004012C0E826F3EEC0BF091
:102C20000101200E006F000E016F000E026F000EFA
:102C3000036FAFEC2AF031C182F40401300E822719
:102C40003EEC0BF032C182F40401300E82273EECE0
:102C50000BF033C182F40401300E82273EEC0BF0FE
:102C6000079471EF1BF00784F5EC34F00CEC2BF0BB
:102C70002DC500F1AFEC2AF004014C0E826F3EEC42
:102C80000BF00401300E826F3EEC0BF004012C0EB1
:102C9000826F3EEC0BF031C182F40401300E8227CA
:102CA0003EEC0BF032C182F40401300E82273EEC80
:102CB0000BF033C182F40401300E82273EEC0BF09E
:102CC00004012C0E826F3EEC0BF00CEC2BF02EC5A9
:102CD00000F1AFEC2AF031C182F40401300E8227FA
:102CE0003EEC0BF032C182F40401300E82273EEC40
:102CF0000BF033C182F40401300E82273EEC0BF05E
:102D0000079471EF1BF004014C0E826F3EEC0BF048
:102D10000401650E826F3EEC0BF004EC2FF071EFB6
:102D20001BF004014C0E826F3EEC0BF00401450ECB
:102D3000826F3EEC0BF021EC2FF071EF1BF00401E1
:102D40004C0E826F3EEC0BF00401620E826F3EEC83
:102D50000BF05BEC2FF071EF1BF004014C0E826F57
:102D60003EEC0BF00401420E826F3EEC0BF03EECA9
:102D70002FF071EF1BF004014C0E826F3EEC0BF054
:102D800004015A0E826F3EEC0BF004012C0E826F90
:102D90003EEC0BF0F5EC34F00CEC2BF005012E5171
:102DA000130A06E005012E51170A0DE0ECEF16F0AC
:102DB0000101000E006F000E016F100E026F000E79
:102DC000036FECEF16F00101000E006F000E016FB3
:102DD000000E026F010E036F0101200E046F000E42
:102DE000056F000E066F000E076F42EC2AF0AFEC85
:102DF0002AF02AC182F40401300E82273EEC0BF047
:102E00002BC182F40401300E82273EEC0BF02CC162
:102E100082F40401300E82273EEC0BF02DC182F4C7
:102E20000401300E82273EEC0BF02EC182F4040127
:102E3000300E82273EEC0BF02FC182F40401300EDD
:102E400082273EEC0BF030C182F40401300E822761
:102E50003EEC0BF031C182F40401300E82273EECCF
:102E60000BF032C182F40401300E82273EEC0BF0ED
:102E700033C182F40401300E82273EEC0BF071EF77
:102E80001BF0078404014C0E826F3EEC0BF0040132
:102E9000310E826F3EEC0BF004012C0E826F3EEC83
:102EA0000BF025C500F126C501F127C502F128C5A3
:102EB00003F10101200E046F000E056F000E066F76
:102EC000000E076F42EC2AF0AFEC2AF02AC182F420
:102ED0000401300E82273EEC0BF02BC182F404017A
:102EE000300E82273EEC0BF02CC182F40401300E30
:102EF00082273EEC0BF02DC182F40401300E8227B4
:102F00003EEC0BF02EC182F40401300E82273EEC21
:102F10000BF02FC182F40401300E82273EEC0BF03F
:102F200030C182F40401300E82273EEC0BF031C137
:102F300082F40401300E82273EEC0BF032C182F4A1
:102F40000401300E82273EEC0BF033C182F4040101
:102F5000300E82273EEC0BF0079471EF1BF00784D4
:102F600004014C0E826F3EEC0BF00401320E826FB6
:102F70003EEC0BF053EC31F0079471EF1BF007843B
:102F800004014C0E826F3EEC0BF00401330E826F95
:102F90003EEC0BF0B0EC31F007944CEF17F00784E7
:102FA00004014C0E826F3EEC0BF00401340E826F74
:102FB0003EEC0BF004012C0E826F3EEC0BF04DEC5E
:102FC0002BF084C32AF185C32BF186C32CF187C370
:102FD0002DF188C32EF189C32FF18AC330F18BC341
:102FE00031F18CC332F18DC333F10101296B5AECFD
:102FF0002BF0D1EC2AF0200E046F000E056F000EAE
:10300000066F000E076F22EC2AF000C121F501C106
:1030100022F502C123F503C124F5A8EC34F034C530
:10302000ABF535C5ACF536C5ADF537C5AEF538C52C
:10303000AFF539C5B0F53AC5B1F55DEC14F0040152
:103040002C0E826F3EEC0BF03BC500F13CC501F14C
:103050003DC502F13EC503F10101000E046F000EF3
:10306000056F010E066F000E076F42EC2AF0AFEC01
:103070002AF029673EEF18F043EF18F004012D0EF7
:10308000826F3EEC0BF030C182F40401300E8227D7
:103090003EEC0BF031C182F40401300E82273EEC8D
:1030A0000BF004012E0E826F3EEC0BF032C182F465
:1030B0000401300E82273EEC0BF033C182F4040190
:1030C000300E82273EEC0BF004012C0E826F3EEC9A
:1030D0000BF00CEC2BF03FC500F140C501F188EC82
:1030E00024F004012C0E826F3EEC0BF00CEC2BF064
:1030F00041C500F1AFEC2AF031C182F40401300E79
:1031000082273EEC0BF032C182F40401300E82279C
:103110003EEC0BF033C182F40401300E82273EEC0A
:103120000BF004012C0E826F3EEC0BF00101036BDF
:10313000026B48C501F147C500F101AFA5EF18F0DA
:103140000101FF0E026FFF0E036FAFEC2AF029673B
:10315000ACEF18F0B1EF18F004012D0E826F3EECC9
:103160000BF02FC182F40401300E82273EEC0BF0ED
:1031700030C182F40401300E82273EEC0BF031C1E5
:1031800082F40401300E82273EEC0BF032C182F44F
:103190000401300E82273EEC0BF033C182F40401AF
:1031A000300E82273EEC0BF004012C0E826F3EECB9
:1031B0000BF00101036B026B4AC501F149C500F137
:1031C00001AFE8EF18F00101FF0E026FFF0E036F71
:1031D000AFEC2AF02967EFEF18F0F4EF18F00401D4
:1031E0002D0E826F3EEC0BF02FC182F40401300EE5
:1031F00082273EEC0BF030C182F40401300E8227AE
:103200003EEC0BF031C182F40401300E82273EEC1B
:103210000BF032C182F40401300E82273EEC0BF039
:1032200033C182F40401300E82273EEC0BF004011E
:103230002C0E826F3EEC0BF00101036B026B4CC550
:1032400001F14BC500F101AF2BEF19F00101FF0EA9
:10325000026FFF0E036FAFEC2AF0296732EF19F00F
:1032600037EF19F004012D0E826F3EEC0BF02FC1E9
:1032700082F40401300E82273EEC0BF030C182F460
:103280000401300E82273EEC0BF031C182F40401C0
:10329000300E82273EEC0BF032C182F40401300E76
:1032A00082273EEC0BF033C182F40401300E8227FA
:1032B0003EEC0BF004012C0E826F3EEC0BF0010192
:1032C000036B026B4EC501F14DC500F101AF6EEF0E
:1032D00019F00101FF0E026FFF0E036FAFEC2AF031
:1032E000296775EF19F07AEF19F004012D0E826F3E
:1032F0003EEC0BF02FC182F40401300E82273EEC2D
:103300000BF030C182F40401300E82273EEC0BF04A
:1033100031C182F40401300E82273EEC0BF032C141
:1033200082F40401300E82273EEC0BF033C182F4AC
:103330000401300E82273EEC0BF004012C0E826F4C
:103340003EEC0BF00101036B026B50C501F14FC560
:1033500000F101AFB1EF19F00101FF0E026FFF0E96
:10336000036FAFEC2AF02967B8EF19F0BDEF19F041
:1033700004012D0E826F3EEC0BF02FC182F404018C
:10338000300E82273EEC0BF030C182F40401300E87
:1033900082273EEC0BF031C182F40401300E82270B
:1033A0003EEC0BF032C182F40401300E82273EEC79
:1033B0000BF033C182F40401300E82273EEC0BF097
:1033C00004012C0E826F3EEC0BF00101036B026BCB
:1033D00052C501F151C500F101AFF4EF19F001013F
:1033E000FF0E026FFF0E036FAFEC2AF02967FBEFB1
:1033F00019F000EF1AF004012D0E826F3EEC0BF075
:103400002FC182F40401300E82273EEC0BF030C154
:1034100082F40401300E82273EEC0BF031C182F4BD
:103420000401300E82273EEC0BF032C182F404011D
:10343000300E82273EEC0BF033C182F40401300ED3
:1034400082273EEC0BF004012C0E826F3EEC0BF059
:103450000101036B026B46C501F145C500F101AFE7
:1034600037EF1AF00101FF0E026FFF0E036FAFEC92
:103470002AF029673EEF1AF043EF1AF004012D0EEF
:10348000826F3EEC0BF02FC182F40401300E8227D4
:103490003EEC0BF030C182F40401300E82273EEC8A
:1034A0000BF031C182F40401300E82273EEC0BF0A8
:1034B00032C182F40401300E82273EEC0BF033C19E
:1034C00082F40401300E82273EEC0BF0079471EF7A
:1034D0001BF04DEC2BF085C32AF186C32BF187C37B
:1034E0002CF188C32DF189C32EF18AC32FF18BC330
:1034F00030F18CC331F18DC332F18EC333F1010150
:10350000296B5AEC2BF0D1EC2AF00101010E046F6B
:10351000000E056F000E066F000E076F11EC2AF00B
:10352000100E046F000E056F000E066F000E076F81
:1035300022EC2AF000C129F501C12AF502C12BF5C0
:1035400003C12CF5DAEC30F004014C0E826F3EEC36
:103550000BF00401460E826F3EEC0BF004012C0EC2
:10356000826F3EEC0BF025C500F126C501F127C5A1
:1035700002F128C503F10101100E046F000E056F62
:10358000000E066F000E076F42EC2AF0AFEC2AF037
:103590002AC182F40401300E82273EEC0BF02BC1CD
:1035A00082F40401300E82273EEC0BF02CC182F431
:1035B0000401300E82273EEC0BF02DC182F4040191
:1035C000300E82273EEC0BF02EC182F40401300E47
:1035D00082273EEC0BF02FC182F40401300E8227CB
:1035E0003EEC0BF030C182F40401300E82273EEC39
:1035F0000BF031C182F40401300E82273EEC0BF057
:1036000032C182F40401300E82273EEC0BF033C14C
:1036100082F40401300E82273EEC0BF071EF1BF0B8
:103620000F98B0EC31F05EEF23F004014C0E826F86
:103630003EEC0BF00401350E826F3EEC0BF0040102
:103640002C0E826F3EEC0BF00CEC2BF00784B5C512
:1036500000F10794AFEC2AF031C182F40401300E7E
:1036600082273EEC0BF032C182F40401300E822737
:103670003EEC0BF033C182F40401300E82273EECA5
:103680000BF071EF1BF073EC31F00CEC2BF033C549
:1036900000F1AFEC2AF004014C0E826F3EEC0BF00F
:1036A0000401360E826F3EEC0BF004012C0E826F8B
:1036B0003EEC0BF031C182F40401300E82273EEC67
:1036C0000BF032C182F40401300E82273EEC0BF085
:1036D00033C182F40401300E82273EEC0BF071EF0F
:1036E0001BF048EC0BF05EEF23F004014C0E826FF0
:1036F0003EEC0BF00401500E826F3EEC0BF0040127
:103700002C0E826F3EEC0BF085C32AF186C32BF1A1
:1037100087C32CF188C32DF189C32EF18AC32FF101
:103720008BC330F18CC331F18DC332F18EC333F1D1
:1037300001015AEC2BF0D1EC2AF003018451530A19
:103740000DE0030184514D0A38E00401780E826FC8
:103750003EEC0BF048EC0BF05EEF23F00401530E4F
:10376000826F3EEC0BF0250E0C6E00C10BF0F9ECF5
:1037700007F0260E0C6E01C10BF0F9EC07F0270ED6
:103780000C6E02C10BF0F9EC07F0280E0C6E03C1B1
:103790000BF0F9EC07F000C153F501C154F502C17B
:1037A00055F503C156F500C157F501C158F502C1E1
:1037B00059F503C15AF552EF1CF004014D0E826F0A
:1037C0003EEC0BF0290E0C6E00C10BF0F9EC07F08B
:1037D00000C15BF500C15CF552EF1CF004014C0E1A
:1037E000826F3EEC0BF00401540E826F3EEC0BF046
:1037F00004012C0E826F3EEC0BF084C32AF185C3CA
:103800002BF186C32CF187C32DF188C32EF189C318
:103810002FF18AC330F18BC331F18DC332F18EC3E6
:1038200033F101015AEC2BF0D1EC2AF00101000E2A
:10383000046F000E056F010E066F000E076F22EC7D
:103840002AF0210E0C6E00C10BF0F9EC07F0220EED
:103850000C6E01C10BF0F9EC07F0230E0C6E02C1E7
:103860000BF0F9EC07F0240E0C6E03C10BF0F9EC31
:1038700007F000C15DF501C15EF502C15FF503C14E
:1038800060F552EF1CF004014C0E826F3EEC0BF021
:103890000401490E826F3EEC0BF004012C0E826F86
:1038A0003EEC0BF0250E10EC08F0E8CF00F1260EF0
:1038B00010EC08F0E8CF01F1270E10EC08F0E8CF8B
:1038C00002F1280E10EC08F0E8CF03F1AFEC2AF07B
:1038D00092EC28F00401730E826F3EEC0BF00401B1
:1038E0002C0E826F3EEC0BF00CEC2BF0290E10EC42
:1038F00008F0E8CF00F1AFEC2AF092EC28F00401D8
:10390000730E826F3EEC0BF004012C0E826F3EECC6
:103910000BF057C500F158C501F159C502F15AC560
:1039200003F1AFEC2AF092EC28F00401730E826FE1
:103930003EEC0BF004012C0E826F3EEC0BF00CEC15
:103940002BF05CC500F1AFEC2AF092EC28F00401FA
:103950006D0E826F3EEC0BF004012C0E826F3EEC7C
:103960000BF05DC500F15EC501F15FC502F160C5F8
:1039700003F179EC23F004012C0E826F3EEC0BF086
:1039800048EC0BF05EEF23F083C32AF184C32BF1E4
:1039900085C32CF186C32DF187C32EF188C32FF187
:1039A00089C330F18AC331F18BC332F18CC333F157
:1039B00001015AEC2BF0D1EC2AF0160E0C6E00C16E
:1039C0000BF0F9EC07F0170E0C6E01C10BF0F9ECDF
:1039D00007F0180E0C6E02C10BF0F9EC07F0190E8F
:1039E0000C6E03C10BF0F9EC07F000C18AF101C1C4
:1039F0008BF102C18CF103C18DF100C18EF101C1C7
:103A00008FF102C190F103C191F1A6EF1DF083C3C4
:103A10002AF184C32BF185C32CF186C32DF187C312
:103A20002EF188C32FF189C330F18AC331F18BC3E2
:103A300032F18CC333F101015AEC2BF0D1EC2AF0B6
:103A400000C18AF101C18BF102C18CF103C18DF17A
:103A500000C18EF101C18FF102C190F103C191F15A
:103A6000A6EF1DF083C32AF184C32BF185C32CF18B
:103A700086C32DF187C32EF188C32FF189C330F19E
:103A80008AC331F18CC332F18DC333F101015AEC99
:103A90002BF0D1EC2AF00101000E046F000E056F2F
:103AA000010E066F000E076F22EC2AF01A0E0C6E44
:103AB00000C10BF0F9EC07F01B0E0C6E01C10BF00E
:103AC000F9EC07F01C0E0C6E02C10BF0F9EC07F0DC
:103AD0001D0E0C6E03C10BF0F9EC07F000C192F162
:103AE00001C193F102C194F103C195F1A6EF1DF05C
:103AF00083C32AF184C32BF185C32CF186C32DF136
:103B000087C32EF188C32FF189C330F18AC331F105
:103B10008CC332F18DC333F101015AEC2BF0D1EC9F
:103B20002AF00101000E046F000E056F010E066FF2
:103B3000000E076F22EC2AF000C192F101C193F14F
:103B400002C194F103C195F1A6EF1DF0160E10EC21
:103B500008F0E8CF00F1170E10EC08F0E8CF01F103
:103B6000180E10EC08F0E8CF02F1190E10EC08F076
:103B7000E8CF03F1AFEC2AF092EC28F00401730EC9
:103B8000826F3EEC0BF004012C0E826F3EEC0BF0CA
:103B90008AC100F18BC101F18CC102F18DC103F129
:103BA000AFEC2AF092EC28F00401730E826F3EEC29
:103BB0000BF004012C0E826F3EEC0BF01A0E10EC91
:103BC00008F0E8CF00F11B0E10EC08F0E8CF01F18F
:103BD0001C0E10EC08F0E8CF02F11D0E10EC08F0FE
:103BE000E8CF03F179EC23F004012C0E826F3EEC58
:103BF0000BF092C100F193C101F194C102F195C1A2
:103C000003F179EC23F048EC0BF05EEF23F00401B4
:103C1000690E826F3EEC0BF004012C0E826F3EECBD
:103C20000BF00101040E006F000E016F000E026F19
:103C3000000E036FAFEC2AF02CC182F40401300EA9
:103C400082273EEC0BF02DC182F40401300E822756
:103C50003EEC0BF02EC182F40401300E82273EECC4
:103C60000BF02FC182F40401300E82273EEC0BF0E2
:103C700030C182F40401300E82273EEC0BF031C1DA
:103C800082F40401300E82273EEC0BF032C182F444
:103C90000401300E82273EEC0BF033C182F40401A4
:103CA000300E82273EEC0BF004012C0E826F3EECAE
:103CB0000BF001010B0E006F000E016F000E026F82
:103CC000000E036FAFEC2AF02CC182F40401300E19
:103CD00082273EEC0BF02DC182F40401300E8227C6
:103CE0003EEC0BF02EC182F40401300E82273EEC34
:103CF0000BF02FC182F40401300E82273EEC0BF052
:103D000030C182F40401300E82273EEC0BF031C149
:103D100082F40401300E82273EEC0BF032C182F4B3
:103D20000401300E82273EEC0BF033C182F4040113
:103D3000300E82273EEC0BF004012C0E826F3EEC1D
:103D40000BF00101240E006F000E016F000E026FD8
:103D5000000E036FAFEC2AF02CC182F40401300E88
:103D600082273EEC0BF02DC182F40401300E822735
:103D70003EEC0BF02EC182F40401300E82273EECA3
:103D80000BF02FC182F40401300E82273EEC0BF0C1
:103D900030C182F40401300E82273EEC0BF031C1B9
:103DA00082F40401300E82273EEC0BF032C182F423
:103DB0000401300E82273EEC0BF033C182F4040183
:103DC000300E82273EEC0BF004012C0E826F3EEC8D
:103DD0000BF0200EF86EF76AF66A04010900F5CFC1
:103DE00082F43EEC0BF00900F5CF82F43EEC0BF0D0
:103DF0000900F5CF82F43EEC0BF00900F5CF82F418
:103E00003EEC0BF00900F5CF82F43EEC0BF009001C
:103E1000F5CF82F43EEC0BF00900F5CF82F43EECD6
:103E20000BF00900F5CF82F43EEC0BF048EC0BF000
:103E30005EEF23F08351630AD8A45EEF23F0845130
:103E4000610AD8A45EEF23F085516C0AD8A45EEF16
:103E500023F08651410A42E08651440A1BE0865114
:103E6000420AD8B481EF1FF08651350AD8B4E8EF82
:103E700024F08651360AD8B43DEF25F08651370A32
:103E8000D8B4A6EF25F08651380AD8B404EF26F04E
:103E90005EEF23F00798079A04017A0E826F3EECDA
:103EA0000BF00401780E826F3EEC0BF00401640EFF
:103EB000826F3EEC0BF081A865EF1FF00401550EF8
:103EC000826F3EEC0BF06AEF1FF004014C0E826F24
:103ED0003EEC0BF048EC0BF05EEF23F00788079AFE
:103EE00004017A0E826F3EEC0BF00401410E826FEA
:103EF0003EEC0BF00401610E826F3EEC0BF05BEFC9
:103F00001FF00798078A04017A0E826F3EEC0BF0CF
:103F10000401420E826F3EEC0BF00401610E826FD1
:103F20003EEC0BF05BEF1FF0010166679FEF1FF0A7
:103F300067679FEF1FF068679FEF1FF06967B7EF34
:103F40001FF04F67ABEF1FF05067ABEF1FF05167EB
:103F5000ABEF1FF05267B7EF1FF00101000E006FCB
:103F6000000E016F000E026F000E036F12000101C0
:103F7000620E046F010E056F000E066F000E076FD4
:103F800066C100F167C101F168C102F169C103F1C5
:103F900011EC2AF003BF3BEF20F00101000E046F8B
:103FA000A80E056F550E066F020E076F66C100F171
:103FB00067C101F168C102F169C103F166C186F10F
:103FC00067C187F168C188F169C189F111EC2AF0F4
:103FD00003BFF4EF1FF00101000E866FA80E876F7C
:103FE000550E886F020E896F0E0E10EC08F0E8CFA8
:103FF00018F10F0E10EC08F0E8CF19F1100E10ECCC
:1040000008F0E8CF1AF1110E10EC08F0E8CF1BF120
:104010005AEC29F086C104F187C105F188C106F187
:1040200089C107F111EC2AF007821EEC29F05AEC45
:1040300029F007921EEC29F086C100F187C101F139
:1040400088C102F189C103F107921EEC29F0CC0E60
:10405000046FE00E056F870E066F050E076F11ECFB
:104060002AF000C118F101C119F102C11AF103C10E
:104070001BF173EF20F00101800E006F1A0E016F2B
:10408000060E026F000E036F4FC104F150C105F11F
:1040900051C106F152C107F111EC2AF003AF54EF00
:1040A00020F00CEC2BF012000E0E10EC08F0E8CF14
:1040B00018F10F0E10EC08F0E8CF19F1100E10EC0B
:1040C00008F0E8CF1AF1110E10EC08F0E8CF1BF160
:1040D0004FC100F150C101F151C102F152C103F1D0
:1040E00007821EEC29F018C100F119C101F11AC1B3
:1040F00002F11BC103F112000401730E826F3EEC4A
:104100000BF004012C0E826F3EEC0BF0078462C1B1
:1041100066F163C167F164C168F165C169F14BC1C2
:104120004FF14CC150F14DC151F14EC152F157C147
:1041300059F158C15AF10794A2EC20F048EC0BF069
:104140005EEF23F066C100F167C101F168C102F1C1
:1041500069C103F10101AFEC2AF092EC28F00401EF
:10416000630E826F3EEC0BF004012C0E826F3EEC6E
:104170000BF04FC100F150C101F151C102F152C128
:1041800003F10101AFEC2AF092EC28F00401660E75
:10419000826F3EEC0BF004012C0E826F3EEC0BF0B4
:1041A0000CEC2BF059C100F15AC101F10101AFEC47
:1041B0002AF092EC28F00401740E826F3EEC0BF0B2
:1041C000120010820401530E826F3EEC0BF00401CA
:1041D0002C0E826F3EEC0BF083C32AF184C32BF1CB
:1041E00085C32CF186C32DF187C32EF188C32FF12F
:1041F00089C330F18AC331F18BC332F18CC333F1FF
:1042000001015AEC2BF0D1EC2AF000C166F101C19A
:1042100067F102C168F103C169F18EC32AF18FC34E
:104220002BF190C32CF191C32DF192C32EF193C3C6
:104230002FF194C330F195C331F196C332F197C396
:1042400033F101015AEC2BF0D1EC2AF000C14FF10F
:1042500001C150F102C151F103C152F14DEC2BF0FB
:1042600099C32FF19AC330F19BC331F19CC332F152
:104270009DC333F101015AEC2BF0D1EC2AF000C1BF
:1042800059F101C15AF1A2EC20F004012C0E826F09
:104290003EEC0BF053EF21F08251520A03E10F8202
:1042A00053EF21F00F928251750A03E110845AEF07
:1042B00021F010948251550A03E1108661EF21F03C
:1042C0001096078410B2BEEF21F010A4AAEF21F0DF
:1042D000B6C166F1B7C167F1B8C168F1B9C169F19A
:1042E000BAC16AF1BBC16BF1BCC16CF1BDC16DF16A
:1042F000BEC16EF1BFC16FF1C0C170F1C1C171F13A
:10430000C2C172F1C3C173F1C4C174F1C5C175F109
:10431000C6C176F1C7C177F1C8C178F1C9C179F1D9
:10432000CAC17AF1CBC17BF1CCC17CF1CDC17DF1A9
:10433000CEC17EF1CFC17FF1D0C180F1D1C181F179
:10434000D2C182F1D3C183F1D4C184F1D5C185F149
:10435000B2EF21F062C166F163C167F164C168F137
:1043600065C169F14BC14FF14CC150F14DC151F1E3
:104370004EC152F157C159F158C15AF107940FA0DB
:10438000E0EF21F001019267CDEF21F09367CDEFCF
:1043900021F09467CDEF21F09567D1EF21F0E0EFA8
:1043A00021F094EC1FF092C104F193C105F194C186
:1043B00006F195C107F111EC2AF003BF24EF23F0B9
:1043C00094EC1FF00101000E046F000E056F010E4A
:1043D000066F000E076F42EC2AF010A4F7EF21F0F1
:1043E0000401750E826F3EEC0BF0FCEF21F004012E
:1043F000720E826F3EEC0BF004012C0E826F3EECCD
:104400000BF0AFEC2AF029670BEF22F00401200E2D
:10441000826F0EEF22F004012D0E826F3EEC0BF046
:1044200030C182F40401300E82273EEC0BF031C122
:1044300082F40401300E82273EEC0BF004012E0EB4
:10444000826F3EEC0BF032C182F40401300E822701
:104450003EEC0BF033C182F40401300E82273EECB7
:104460000BF004016D0E826F3EEC0BF004012C0E7C
:10447000826F3EEC0BF04FC100F150C101F151C110
:1044800002F152C103F10101AFEC2AF092EC28F0E5
:104490000401480E826F3EEC0BF004017A0E826F2D
:1044A0003EEC0BF004012C0E826F3EEC0BF066C16B
:1044B00000F167C101F168C102F169C103F10101B5
:1044C000AFEC2AF092EC28F00401630E826F3EEC10
:1044D0000BF004012C0E826F3EEC0BF066C100F174
:1044E00067C101F168C102F169C103F101010A0E5E
:1044F000046F000E056F000E066F000E076F22ECB2
:104500002AF0000E046F120E056F000E066F000EEB
:10451000076F42EC2AF0AFEC2AF02AC182F40401C2
:10452000300E82273EEC0BF02BC182F40401300EDA
:1045300082273EEC0BF02CC182F40401300E82275E
:104540003EEC0BF02DC182F40401300E82273EECCC
:104550000BF02EC182F40401300E82273EEC0BF0EA
:104560002FC182F40401300E82273EEC0BF030C1E3
:1045700082F40401300E82273EEC0BF004012E0E73
:10458000826F3EEC0BF031C182F40401300E8227C1
:104590003EEC0BF032C182F40401300E82273EEC77
:1045A0000BF033C182F40401300E82273EEC0BF095
:1045B0000401730E826F3EEC0BF004012C0E826F2F
:1045C0003EEC0BF00CEC2BF059C100F15AC101F19B
:1045D00088EC24F00FB2F0EF22F00FA022EF23F0CE
:1045E00004012C0E826F3EEC0BF0200EF86EF76A81
:1045F000F66A04010900F5CF82F43EEC0BF00900E5
:10460000F5CF82F43EEC0BF00900F5CF82F43EECDE
:104610000BF00900F5CF82F43EEC0BF00900F5CF6A
:1046200082F43EEC0BF00900F5CF82F43EEC0BF087
:104630000900F5CF82F43EEC0BF00900F5CF82F4CF
:104640003EEC0BF048EC0BF00F905EEF23F0040112
:10465000630E826F3EEC0BF004012C0E826F3EEC79
:104660000BF064EC23F004012C0E826F3EEC0BF097
:10467000D7EC23F004012C0E826F3EEC0BF053ECD0
:1046800024F004012C0E826F3EEC0BF00101F80EB9
:10469000006FCD0E016F660E026F030E036F79EC93
:1046A00023F004012C0E826F3EEC0BF069EC24F039
:1046B00048EC0BF05EEF23F048EC0BF00301C26B0B
:1046C000079010926DEF26F0D8900E0E10EC08F0C7
:1046D000E8CF00F10F0E10EC08F0E8CF01F1100E5A
:1046E00010EC08F0E8CF02F1110E10EC08F0E8CF62
:1046F00003F10101000E046F000E056F010E066F3D
:10470000000E076F42EC2AF0AFEC2AF02AC182F4C7
:104710000401300E82273EEC0BF02BC182F4040121
:10472000300E82273EEC0BF02CC182F40401300ED7
:1047300082273EEC0BF02DC182F40401300E82275B
:104740003EEC0BF02EC182F40401300E82273EECC9
:104750000BF02FC182F40401300E82273EEC0BF0E7
:1047600030C182F40401300E82273EEC0BF031C1DF
:1047700082F40401300E82273EEC0BF004012E0E71
:10478000826F3EEC0BF032C182F40401300E8227BE
:104790003EEC0BF033C182F40401300E82273EEC74
:1047A0000BF004016D0E826F3EEC0BF01200120E46
:1047B00010EC08F0E8CF00F1130E10EC08F0E8CF91
:1047C00001F1140E10EC08F0E8CF02F1150E10EC18
:1047D00008F0E8CF03F101010A0E046F000E056F27
:1047E000000E066F000E076F22EC2AF0000E046F19
:1047F000120E056F000E066F000E076F42EC2AF0D6
:10480000AFEC2AF02AC182F40401300E82273EEC7C
:104810000BF02BC182F40401300E82273EEC0BF02A
:104820002CC182F40401300E82273EEC0BF02DC126
:1048300082F40401300E82273EEC0BF02EC182F48C
:104840000401300E82273EEC0BF02FC182F40401EC
:10485000300E82273EEC0BF030C182F40401300EA2
:1048600082273EEC0BF004012E0E826F3EEC0BF023
:1048700031C182F40401300E82273EEC0BF032C1CC
:1048800082F40401300E82273EEC0BF033C182F437
:104890000401300E82273EEC0BF00401730E826F90
:1048A0003EEC0BF012000A0E10EC08F0E8CF00F11D
:1048B0000B0E10EC08F0E8CF01F10C0E10EC08F034
:1048C000E8CF02F10D0E10EC08F0E8CF03F188EF0D
:1048D00024F0060E10EC08F0E8CF00F1070E10EC03
:1048E00008F0E8CF01F1080E10EC08F0E8CF02F173
:1048F000090E10EC08F0E8CF03F188EF24F0010175
:104900000CEC2BF0078457C100F158C101F107945A
:104910000101E80E046F800E056F000E066F000E99
:10492000076F22EC2AF0000E046F040E056F000ED4
:10493000066F000E076F42EC2AF0880E046F130E0C
:10494000056F000E066F000E076F11EC2AF00A0EBD
:10495000046F000E056F000E066F000E076F42EC2D
:104960002AF0AFEC2AF001012967BCEF24F0040122
:10497000200E826FBFEF24F004012D0E826F3EECFB
:104980000BF030C182F40401300E82273EEC0BF0B4
:1049900031C182F40401300E82273EEC0BF032C1AB
:1049A00082F40401300E82273EEC0BF004012E0E3F
:1049B000826F3EEC0BF033C182F40401300E82278B
:1049C0003EEC0BF00401430E826F3EEC0BF0120044
:1049D00087C32AF188C32BF189C32CF18AC32DF137
:1049E0008BC32EF18CC32FF18DC330F18EC331F107
:1049F00090C332F191C333F10101296B5AEC2BF0D2
:104A0000D1EC2AF00101000E046F000E056F010EBB
:104A1000066F000E076F22EC2AF00E0E0C6E00C11E
:104A20000BF0F9EC07F00F0E0C6E01C10BF0F9EC76
:104A300007F0100E0C6E02C10BF0F9EC07F0110E2E
:104A40000C6E03C10BF0F9EC07F004017A0E826FD3
:104A50003EEC0BF004012C0E826F3EEC0BF00401D7
:104A6000350E826F3EEC0BF004012C0E826F3EEC93
:104A70000BF064EC23F06AEF1FF087C32AF188C3C0
:104A80002BF189C32CF18AC32DF18BC32EF18CC37A
:104A90002FF18DC330F18EC331F190C332F191C348
:104AA00033F10101296B5AEC2BF0D1EC2AF0880E7E
:104AB000046F130E056F000E066F000E076F16ECE5
:104AC0002AF0000E046F040E056F000E066F000E34
:104AD000076F22EC2AF00101E80E046F800E056FCB
:104AE000000E066F000E076F42EC2AF00A0E0C6EE5
:104AF00000C10BF0F9EC07F00B0E0C6E01C10BF0CE
:104B0000F9EC07F00C0E0C6E02C10BF0F9EC07F09B
:104B10000D0E0C6E03C10BF0F9EC07F004017A0ED8
:104B2000826F3EEC0BF004012C0E826F3EEC0BF01A
:104B30000401360E826F3EEC0BF004012C0E826FE6
:104B40003EEC0BF053EC24F06AEF1FF087C32AF120
:104B500088C32BF189C32CF18AC32DF18BC32EF1AD
:104B60008CC32FF18DC330F18FC331F190C332F17B
:104B700091C333F101015AEC2BF0D1EC2AF0000E75
:104B8000046F120E056F000E066F000E076F22EC09
:104B90002AF001010A0E046F000E056F000E066F69
:104BA000000E076F42EC2AF0120E0C6E00C10BF0E3
:104BB000F9EC07F0130E0C6E01C10BF0F9EC07F0E5
:104BC000140E0C6E02C10BF0F9EC07F0150E0C6E12
:104BD00003C10BF0F9EC07F004017A0E826F3EEC92
:104BE0000BF004012C0E826F3EEC0BF00401370E2B
:104BF000826F3EEC0BF004012C0E826F3EEC0BF04A
:104C0000D7EC23F06AEF1FF087C32AF188C32BF19A
:104C100089C32CF18AC32DF18BC32EF18CC32FF1E4
:104C20008DC330F18EC331F190C332F191C333F1B2
:104C30000101296B5AEC2BF0D1EC2AF0880E046F9D
:104C4000130E056F000E066F000E076F16EC2AF0AC
:104C5000000E046F040E056F000E066F000E076F46
:104C600022EC2AF00101E80E046F800E056F000EA1
:104C7000066F000E076F42EC2AF0060E0C6E00C1A4
:104C80000BF0F9EC07F0070E0C6E01C10BF0F9EC1C
:104C900007F0080E0C6E02C10BF0F9EC07F0090EDC
:104CA0000C6E03C10BF0F9EC07F004017A0E826F71
:104CB0003EEC0BF004012C0E826F3EEC0BF0040175
:104CC000380E826F3EEC0BF004012C0E826F3EEC2E
:104CD0000BF069EC24F06AEF1FF081A82BEF27F0AE
:104CE00007A8E4EF26F00101800E006F1A0E016F95
:104CF000060E026F000E036F4BC104F14CC105F1AB
:104D00004DC106F14EC107F111EC2AF003BF2BEFA4
:104D100027F08CEC28F04BC100F14CC101F14DC1E2
:104D200002F14EC103F107821EEC29F018C104F113
:104D300019C105F11AC106F11BC107F1F80E006F88
:104D4000CD0E016F660E026F030E036F11EC2AF099
:104D50000E0E0C6E00C10BF0F9EC07F00F0E0C6E8E
:104D600001C10BF0F9EC07F0100E0C6E02C10BF054
:104D7000F9EC07F0110E0C6E03C10BF0F9EC07F023
:104D8000078401010CEC2BF057C100F158C101F16F
:104D900007940A0E0C6E00C10BF0F9EC07F00B0E35
:104DA0000C6E01C10BF0F9EC07F00C0E0C6E02C199
:104DB0000BF0F9EC07F00D0E0C6E03C10BF0F9ECE3
:104DC00007F007982BEF27F007AA2BEF27F00784AF
:104DD00001010CEC2BF057C100F158C101F107940F
:104DE000060E0C6E00C10BF0F9EC07F0070E0C6E0E
:104DF00001C10BF0F9EC07F0080E0C6E02C10BF0CC
:104E0000F9EC07F0090E0C6E03C10BF0F9EC07F09A
:104E1000078462C100F163C101F164C102F165C19F
:104E200003F10794120E0C6E00C10BF0F9EC07F0C1
:104E3000130E0C6E01C10BF0F9EC07F0140E0C6EA2
:104E400002C10BF0F9EC07F0150E0C6E03C10BF06C
:104E5000F9EC07F0079A0401805181197F0B0BE0F0
:104E60009EA809D014EE00F081517F0BE126E75097
:104E7000812B0F01AD6E05012F51010A13E081AAAC
:104E800052EF27F005012F51000A0AE00FB852EF48
:104E900027F00501306752EF27F00FB852EF27F0E7
:104EA00034EF35F081B867EF27F075EC2DF0050190
:104EB0002F51020A02E067EF27F05C2F67EF27F01F
:104EC0005BC55CF50501010E306F3C0E316F9DEF47
:104ED0000AF006013251385D3351D8A0010F395D17
:104EE000800BD8A478EF27F032C638F633C639F6EF
:104EF000120006013251365D3351D8A0010F375DE3
:104F0000800BD8B488EF27F032C636F633C637F6B2
:104F1000120007841AC632F61BC633F61CC638F6D2
:104F20001DC639F669EC27F01EC632F61FC633F6E9
:104F300069EC27F020C632F621C633F669EC27F07B
:104F40001AC632F61BC633F61CC636F61DC637F631
:104F500079EC27F01EC632F61FC633F679EC27F03F
:104F600020C632F621C633F679EC27F03851365F89
:104F70003951D8A03929375F0CEC2BF036C600F137
:104F800037C601F118EC2BF000C13AF601C13BF62F
:104F900022C632F623C633F624C638F625C639F6BD
:104FA00069EC27F026C632F627C633F669EC27F0FF
:104FB00028C632F629C633F669EC27F022C632F647
:104FC00023C633F624C636F625C637F679EC27F025
:104FD00026C632F627C633F679EC27F028C632F615
:104FE00029C633F679EC27F03851365F3951D8A00D
:104FF0003929375F0CEC2BF036C600F137C601F1CA
:1050000018EC2BF000C13CF601C13DF62AC632F681
:105010002BC633F62CC638F62DC639F669EC27F0C8
:105020002EC632F62FC633F669EC27F030C632F6BC
:1050300031C633F669EC27F02AC632F62BC633F6B2
:105040002CC636F62DC637F679EC27F02EC632F68A
:105050002FC633F679EC27F030C632F631C633F678
:1050600079EC27F03851365F3951D8A03929375FAC
:105070000CEC2BF036C600F137C601F118EC2BF022
:1050800000C13EF601C13FF63AC632F63BC633F6E2
:105090003CC636F63DC637F679EC27F03EC632F60A
:1050A0003FC633F679EC27F00794120018C100F1DF
:1050B00019C101F11AC102F11BC103F1000E046F05
:1050C000000E056F010E066F000E076F42EC2AF00E
:1050D00029A181EF28F02051D8B481EF28F018C120
:1050E00000F119C101F11AC102F11BC103F1000E57
:1050F000046F000E056F0A0E066F000E076F42EC7C
:105100002AF0120001010451001305510113065148
:1051100002130751031312000101186B196B1A6B6C
:105120001B6B12002AC182F40401300E82273EEC70
:105130000BF02BC182F40401300E82273EEC0BF001
:105140002CC182F40401300E82273EEC0BF02DC1FD
:1051500082F40401300E82273EEC0BF02EC182F463
:105160000401300E82273EEC0BF02FC182F40401C3
:10517000300E82273EEC0BF030C182F40401300E79
:1051800082273EEC0BF031C182F40401300E8227FD
:105190003EEC0BF032C182F40401300E82273EEC6B
:1051A0000BF033C182F40401300E82273EEC0BF089
:1051B00012002FC182F40401300E82273EEC0BF066
:1051C00030C182F40401300E82273EEC0BF031C175
:1051D00082F40401300E82273EEC0BF032C182F4DF
:1051E0000401300E82273EEC0BF033C182F404013F
:1051F000300E82273EEC0BF01200060E116E060EEA
:10520000126E060E136E112E03EF29F0122E03EF0D
:1052100029F0132E03EF29F08B84020E116E020E7B
:10522000126E020E136E112E13EF29F0122E13EFD1
:1052300029F0132E13EF29F08B9412000101005373
:1052400005E1015303E1025301E1002BE1EC29F0F8
:105250000CEC2BF03951006F3A51016F420E046F84
:105260004B0E056F000E066F000E076F22EC2AF042
:1052700000C104F101C105F102C106F103C107F14A
:1052800018C100F119C101F11AC102F11BC103F1EA
:1052900007B24FEF29F016EC2AF051EF29F011EC8C
:1052A0002AF000C118F101C119F102C11AF103C1BC
:1052B0001BF112000CEC2BF059C100F15AC101F1A5
:1052C000060E10EC08F0E8CF04F1070E10EC08F021
:1052D000E8CF05F1080E10EC08F0E8CF06F1090E52
:1052E00010EC08F0E8CF07F111EC2AF000C124F12E
:1052F00001C125F102C126F103C127F1290E046F76
:10530000000E056F000E066F000E076F22EC2AF0EC
:10531000EE0E046F430E056F000E066F000E076F52
:1053200016EC2AF024C104F125C105F126C106F1CD
:1053300027C107F122EC2AF000C11CF101C11DF1C7
:1053400002C11EF103C11FF1120E10EC08F0E8CFEC
:1053500004F1130E10EC08F0E8CF05F1140E10EC78
:1053600008F0E8CF06F1150E10EC08F0E8CF07F1D1
:105370000D0E006F000E016F000E026F000E036F26
:1053800022EC2AF0180E046F000E056F000E066F57
:10539000000E076F42EC2AF01CC104F11DC105F19B
:1053A0001EC106F11FC107F116EC2AF06A0E046F48
:1053B0002A0E056F000E066F000E076F11EC2AF023
:1053C0001200BF0EFA6E200E3A6F396BD89000377C
:1053D000013702370337D8B0F2EF29F03A2FE7EF61
:1053E00029F039073A070353D8B412000331070BE9
:1053F00080093F6F03390F0B010F396F80EC5FF0AD
:10540000406F390580EC5FF0405D405F396B3F33A2
:10541000D8B0392739333FA907EF2AF0405139274F
:105420001200010131EC2BF0D8B012000101035140
:105430000719346FF4EC2AF0D8900751031934AFF0
:10544000800F12000101346B18EC2BF0D8A02EEC69
:105450002BF0D8B0120003EC2BF00CEC2BF01F0E4D
:10546000366F44EC2BF00B35D8B0F4EC2AF0D8A012
:105470000335D8B01200362F31EF2AF034B11BECCF
:105480002BF012000101346B0451051106110711B4
:105490000008D8A018EC2BF0D8A02EEC2BF0D8B038
:1054A0001200086B096B0A6B0B6B44EC2BF01F0EA0
:1054B000366F44EC2BF007510B5DD8A46CEF2AF04B
:1054C00006510A5DD8A46CEF2AF00551095DD8A4F5
:1054D0006CEF2AF00451085DD8A07FEF2AF0045148
:1054E000085F0551D8A0053D095F0651D8A0063DCB
:1054F0000A5F0751D8A0073D0B5FD8900081362F77
:1055000059EF2AF034B11BEC2BF0346B18EC2BF074
:10551000D89048EC2BF007510B5DD8A49CEF2AF0F3
:1055200006510A5DD8A49CEF2AF00551095DD8A464
:105530009CEF2AF00451085DD8A0ABEF2AF0003FA1
:10554000ABEF2AF0013FABEF2AF0023FABEF2AF0BE
:10555000032BD8B4120034B11BEC2BF01200010164
:10556000346B18EC2BF0D8B012004DEC2BF0200E61
:10557000366F003701370237033711EE33F00A0E6A
:10558000376FE7360A0EE75CD8B0E76EE552372F83
:10559000C1EF2AF0362FB9EF2AF034B12981D89023
:1055A000120001010A0E346F200E366F11EE29F041
:1055B0003451376F0A0ED890E652D8B0E726E7325A
:1055C000372FDCEF2AF00333023301330033362F59
:1055D000D6EF2AF0E750FF0FD8A00335D8B012005D
:1055E00029B11BEC2BF01200045100270551D8B053
:1055F000053D01270651D8B0063D02270751D8B016
:10560000073D032712000051086F0151096F025135
:105610000A6F03510B6F12000101006B016B026BEB
:10562000036B12000101046B056B066B076B120024
:105630000335D8A012000351800B001F011F021F69
:10564000031F003F2BEF2BF0013F2BEF2BF0023F0E
:105650002BEF2BF0032B342B032512000735D8A09A
:1056600012000751800B041F051F061F071F043F70
:1056700041EF2BF0053F41EF2BF0063F41EF2BF0C0
:10568000072B342B07251200003701370237033769
:10569000083709370A370B3712000101296B2A6BCB
:1056A0002B6B2C6B2D6B2E6B2F6B306B316B326B2E
:1056B000336B120001012A510F0B2A6F2B510F0B74
:1056C0002B6F2C510F0B2C6F2D510F0B2D6F2E515B
:1056D0000F0B2E6F2F510F0B2F6F30510F0B306FA1
:1056E00031510F0B316F32510F0B326F33510F0BA2
:1056F000336F1200899C000EC76E200EC66E9E96F8
:10570000C69EC50EC96EFF0E9EB602D0E82EFCD70F
:105710009E96C69E000EC96EFF0E9EB602D0E82E63
:10572000FCD7C9CF00F69E96C69E000EC96EFF0E2E
:105730009EB602D0E82EFCD7C9CF01F6898C1200A4
:10574000000EC76E200EC66E899C9E96C69EC80E21
:10575000C96EFF0E9EB602D0E82EFCD79E96C69E5E
:10576000000EC96EFF0E9EB602D0E82EFCD7C9CF40
:1057700002F69E96C69E000EC96EFF0E9EB602D021
:10578000E82EFCD7C9CF03F6898C899C9E96C69ECD
:10579000CA0EC96EFF0E9EB602D0E82EFCD79E96AA
:1057A000C69E000EC96EFF0E9EB602D0E82EFCD734
:1057B000C9CF0AF69E96C69E000EC96EFF0E9EB613
:1057C00002D0E82EFCD7C9CF0BF6898C899C9E9617
:1057D000C69ECC0EC96EFF0E9EB602D0E82EFCD738
:1057E0009E96C69E000EC96EFF0E9EB602D0E82E93
:1057F000FCD7C9CF12F69E96C69E000EC96EFF0E4C
:105800009EB602D0E82EFCD7C9CF13F6898C1200C1
:10581000000EC76E200EC66E899C9E96C69EE80E30
:10582000C96EFF0E9EB602D0E82EFCD79E96C69E8D
:10583000000EC96EFF0E9EB602D0E82EFCD7C9CF6F
:105840001AF69E96C69E000EC96EFF0E9EB602D038
:10585000E82EFCD7C9CF1BF6898C899C9E96C69EE4
:10586000EA0EC96EFF0E9EB602D0E82EFCD79E96B9
:10587000C69E000EC96EFF0E9EB602D0E82EFCD763
:10588000C9CF22F69E96C69E000EC96EFF0E9EB62A
:1058900002D0E82EFCD7C9CF23F6898C899C9E962E
:1058A000C69EEC0EC96EFF0E9EB602D0E82EFCD747
:1058B0009E96C69E000EC96EFF0E9EB602D0E82EC2
:1058C000FCD7C9CF2AF69E96C69E000EC96EFF0E63
:1058D0009EB602D0E82EFCD7C9CF2BF6898C1200D9
:1058E000000EC76E200EC66E899C9E96C69E240E24
:1058F000C96EFF0E9EB602D0E82EFCD79E96C69EBD
:10590000E40EC96EFF0E9EB602D0E82EFCD7898C3D
:10591000899C9E96C69E200EC96EFF0E9EB602D032
:10592000E82EFCD79E96C69E5F0EC96EFF0E9EB6F1
:1059300002D0E82EFCD7898C899C9E96C69E210EAB
:10594000C96EFF0E9EB602D0E82EFCD79E96C69E6C
:10595000C00EC96EFF0E9EB602D0E82EFCD7898C11
:10596000899C9E96C69E260EC96EFF0E9EB602D0DC
:10597000E82EFCD79E96C69E000EC96EFF0E9EB600
:1059800002D0E82EFCD7898C12008984000EC76EE5
:10599000220EC66E9E96C69E000EC96EFF0E9EB665
:1059A00002D0E82EFCD79E96C69E000EC96EFF0E52
:1059B0009EB602D0E82EFCD7C9CFABF59E96C69E08
:1059C000000EC96EFF0E9EB602D0E82EFCD7C9CFDE
:1059D000ACF59E96C69E000EC96EFF0E9EB602D016
:1059E000E82EFCD7C9CFADF59E96C69E000EC96EB7
:1059F000FF0E9EB602D0E82EFCD7C9CFAEF59E961C
:105A0000C69E000EC96EFF0E9EB602D0E82EFCD7D1
:105A1000C9CFAFF59E96C69E000EC96EFF0E9EB60C
:105A200002D0E82EFCD7C9CFB0F59E96C69E000ED8
:105A3000C96EFF0E9EB602D0E82EFCD7C9CFB1F5D5
:105A4000899478EC2FF012008984000EC76E220E24
:105A5000C66E9E96C69E800EC96EFF0E9EB602D082
:105A6000E82EFCD79E96C69EABC5C9FFFF0E9EB61C
:105A700002D0E82EFCD79E96C69EACC5C9FFFF0E8D
:105A80009EB602D0E82EFCD79E96C69EADC5C9FF35
:105A9000FF0E9EB602D0E82EFCD79E96C69EAEC5DF
:105AA000C9FFFF0E9EB602D0E82EFCD79E96C69E7A
:105AB000AFC5C9FFFF0E9EB602D0E82EFCD79E965A
:105AC000C69EB0C5C9FFFF0E9EB602D0E82EFCD719
:105AD0009E96C69EB1C5C9FFFF0E9EB602D0E82EA7
:105AE000FCD7899478EC2FF012008984000EC76EE1
:105AF000220EC66E9E96C69E070EC96EFF0E9EB6FD
:105B000002D0E82EFCD79E96C69E000EC96EFF0EF0
:105B10009EB602D0E82EFCD7C9CFABF59E96C69EA6
:105B2000000EC96EFF0E9EB602D0E82EFCD7C9CF7C
:105B3000ACF59E96C69E000EC96EFF0E9EB602D0B4
:105B4000E82EFCD7C9CFADF59E96C69E000EC96E55
:105B5000FF0E9EB602D0E82EFCD7C9CFAEF58994D1
:105B600078EC2FF08984000EC76E220EC66E9E96CA
:105B7000C69E0F0EC96EFF0E9EB602D0E82EFCD751
:105B80009E96C69E000EC96EFF0E9EB602D0E82EEF
:105B9000FCD7C9CFB3F5899478EC2FF01200898433
:105BA000000EC76E220EC66E9E96C69E870EC96EEA
:105BB000FF0E9EB602D0E82EFCD79E96C69EABC5C1
:105BC000C9FFFF0E9EB602D0E82EFCD79E96C69E59
:105BD000ACC5C9FFFF0E9EB602D0E82EFCD79E963C
:105BE000C69EADC5C9FFFF0E9EB602D0E82EFCD7FB
:105BF0009E96C69EAEC5C9FFFF0E9EB602D0E82E89
:105C0000FCD7899478EC2FF089849E96C69E8F0EDF
:105C1000C96EFF0E9EB602D0E82EFCD79E96C69E99
:105C2000B3C5C9FFFF0E9EB602D0E82EFCD78994FB
:105C300078EC2FF012008984000EC76E220EC66E1B
:105C40009E96C69E870EC96EFF0E9EB602D0E82EA7
:105C5000FCD79E96C69E000EC96EFF0E9EB602D061
:105C6000E82EFCD79E96C69E800EC96EFF0E9EB68D
:105C700002D0E82EFCD79E96C69E800EC96EFF0EFF
:105C80009EB602D0E82EFCD79E96C69E800EC96EA8
:105C9000FF0E9EB602D0E82EFCD7899478EC2FF048
:105CA00089849E96C69E8F0EC96EFF0E9EB602D048
:105CB000E82EFCD79E96C69E010EC96EFF0E9EB6BC
:105CC00002D0E82EFCD7899478EC2FF0120089845A
:105CD000000EC76E220EC66E9E96C69E870EC96EB9
:105CE000FF0E9EB602D0E82EFCD79E96C69E000EF2
:105CF000C96EFF0E9EB602D0E82EFCD79E96C69EB9
:105D0000000EC96EFF0E9EB602D0E82EFCD79E96FE
:105D1000C69E800EC96EFF0E9EB602D0E82EFCD73E
:105D20009E96C69E800EC96EFF0E9EB602D0E82ECD
:105D3000FCD7899478EC2FF089849E96C69E8F0EAE
:105D4000C96EFF0E9EB602D0E82EFCD79E96C69E68
:105D5000010EC96EFF0E9EB602D0E82EFCD78994C4
:105D600078EC2FF012008984000EC76E220EC66EEA
:105D70009E96C69E8F0EC96EFF0E9EB602D0E82E6E
:105D8000FCD778EC2FF09E96C69E810EC96EFF0E52
:105D90009EB602D0E82EFCD7899478EC2FF0898447
:105DA000000EC76E220EC66E9E96C69E8F0EC96EE0
:105DB000FF0E9EB602D0E82EFCD778EC2FF09E9610
:105DC000C69E010EC96EFF0E9EB602D0E82EFCD70D
:105DD000899478EC2FF089849E96C69E910EC96EA8
:105DE000FF0E9EB602D0E82EFCD778EC2FF09E96E0
:105DF000C69EA50EC96EFF0E9EB602D0E82EFCD739
:105E0000899478EC2FF012008984000EC76E220E60
:105E1000C66E9E96C69E8F0EC96EFF0E9EB602D0AF
:105E2000E82EFCD778EC2FF09E96C69E810EC96EA8
:105E3000FF0E9EB602D0E82EFCD7899478EC2FF0A6
:105E400012008984000EC76E220EC66E9E96C69EF4
:105E50008F0EC96EFF0E9EB602D0E82EFCD778ECEE
:105E60002FF09E96C69E010EC96EFF0E9EB602D002
:105E7000E82EFCD7899478EC2FF012008984000E6C
:105E8000C76E220EC66E9E96C69E910EC96EFF0EFE
:105E90009EB602D0E82EFCD778EC2FF09E96C69ED8
:105EA000A50EC96EFF0E9EB602D0E82EFCD78994CF
:105EB00078EC2FF012008984000EC76E220EC66E99
:105EC0009E96C69E910EC96EFF0E9EB602D0E82E1B
:105ED000FCD778EC2FF09E96C69E000EC96EFF0E82
:105EE0009EB602D0E82EFCD7899478EC2FF01200F1
:105EF000050EE82EFED712000501256B266B276BD9
:105F0000286B899A400EC76E200EC66E9E96C69E5E
:105F1000030EC96EFF0E9EB602D0E82EFCD79E96E9
:105F2000C69E27C5C9FFFF0E9EB602D0E82EFCD73D
:105F30009E96C69E26C5C9FFFF0E9EB602D0E82ECD
:105F4000FCD79E96C69E25C5C9FFFF0E9EB602D001
:105F5000E82EFCD79E96C69EC952FF0E9EB602D072
:105F6000E82EFCD7898A0F01C950FF0A01E112000F
:105F700005012E51130A05E005012E51170A0CE008
:105F800012000501E00E256FFF0E266F0F0E276F22
:105F9000000E286FD5EF2FF00501E00E256FFF0EE4
:105FA000266FFF0E276F000E286F899A400EC76E6E
:105FB000200EC66E9E96C69E030EC96EFF0E9EB63E
:105FC00002D0E82EFCD79E96C69E27C5C9FFFF0EBD
:105FD0009EB602D0E82EFCD79E96C69E26C5C9FF67
:105FE000FF0E9EB602D0E82EFCD79E96C69E25C513
:105FF000C9FFFF0E9EB602D0E82EFCD79E96C69E25
:10600000C952FF0E9EB602D0E82EFCD7898A0F0136
:10601000C950FF0A1DE005012E51130A05E00501D4
:106020002E51170A0BE012000501000E256F000E1D
:10603000266F100E276F000E286F12000501000E4C
:10604000256F000E266F000E276F010E286F1200BD
:106050000501256B266B276B286B05012E51130A52
:1060600005E005012E51170A0CE012000501000E93
:10607000216F000E226F080E236F000E246F4AEF6F
:1060800030F00501000E216F000E226F800E236F8D
:10609000000E246F21C500F122C501F123C502F1D4
:1060A00024C503F125C504F126C505F127C506F170
:1060B00028C507F182EC28F000C125F501C126F5BD
:1060C00002C127F503C128F5899A400EC76E200E3C
:1060D000C66E9E96C69E030EC96EFF0E9EB602D079
:1060E000E82EFCD79E96C69E27C5C9FFFF0E9EB61A
:1060F00002D0E82EFCD79E96C69E26C5C9FFFF0E8D
:106100009EB602D0E82EFCD79E96C69E25C5C9FF36
:10611000FF0E9EB602D0E82EFCD79E96C69EC952B0
:10612000FF0E9EB602D0E82EFCD7898AC950FF0A1E
:1061300008E104C125F505C126F506C127F507C10B
:1061400028F5D890050124332333223321332151FC
:10615000E00B216F2167B4EF30F02267B4EF30F02D
:106160002367B4EF30F024674AEF30F00501200ECA
:106170002527E86A2623E86A2723E86A28231200ED
:10618000E86A05012E51130A06E005012E51170A8F
:106190000BE0020E120005012851000A03E127510D
:1061A000F00B07E0010E120005012851000A01E082
:1061B000010E120029C500F12AC501F12BC502F11B
:1061C0002CC503F125C504F126C505F127C506F147
:1061D00028C507F111EC2AF003BF1200C0EC30F023
:1061E000D8A452EF31F0899A400EC76E200EC66EC9
:1061F0009E96C69E060EC96EFF0E9EB602D0E82E73
:10620000FCD7898A899A9E96C69E020EC96EFF0E99
:106210009EB602D0E82EFCD79E96C69E27C5C9FF23
:10622000FF0E9EB602D0E82EFCD79E96C69E26C5CF
:10623000C9FFFF0E9EB602D0E82EFCD79E96C69EE2
:1062400025C5C9FFFF0E9EB602D0E82EFCD79E964C
:10625000C69E000EC96EFF0E9EB602D0E82EFCD779
:10626000898A899A9E96C69E050EC96EFF0E9EB6B5
:1062700002D0E82EFCD79E96C69EC952FF0E9EB64F
:1062800002D0E82EFCD7C9B03BEF31F0898A050176
:10629000200E2527E86A2623E86A2723E86A2823B0
:1062A000DAEF30F01200899A400EC76E200EC66EEB
:1062B0009E96C69E060EC96EFF0E9EB602D0E82EB2
:1062C000FCD7898A899A9E96C69EC70EC96EFF0E14
:1062D0009EB602D0E82EFCD7898A0501256B266B75
:1062E000276B286B1200899A400EC76E200EC66E6F
:1062F0009E96C69E050EC96EFF0E9EB602D0E82E73
:10630000FCD79E96C69EC952FF0E9EB602D0E82EBE
:10631000FCD7C9CF33F5898A1200899A400EC76E1F
:10632000200EC66E9E96C69EB90EC96EFF0E9EB614
:1063300002D0E82EFCD7898A1200899A400EC76ED7
:10634000200EC66E9E96C69EAB0EC96EFF0E9EB602
:1063500002D0E82EFCD7898AFF0EE82EFED7120065
:10636000C0EC30F0D8A41200899A400EC76E200EFF
:10637000C66E9E96C69E030EC96EFF0E9EB602D0D6
:10638000E82EFCD79E96C69E27C5C9FFFF0E9EB677
:1063900002D0E82EFCD79E96C69E26C5C9FFFF0EEA
:1063A0009EB602D0E82EFCD79E96C69E25C5C9FF94
:1063B000FF0E9EB602D0E82EFCD79E96C69EC9520E
:1063C000FF0E9EB602D0E82EFCD7898A0F01C95075
:1063D000FF0AD8A4A7EF34F00501FE0E336FC5EC19
:1063E0002CF0ABC534F5ACC535F5ADC536F5AEC54D
:1063F00037F5AFC538F5B0C539F5B1C53AF50784FD
:10640000B6C166F1B7C167F1B8C168F1B9C169F148
:106410004BC14FF14CC150F14DC151F14EC152F140
:1064200057C159F158C15AF194EC1FF000C13BF526
:1064300001C13CF502C13DF503C13EF505015D67B3
:1064400029EF32F05E6729EF32F05F6729EF32F013
:1064500060672DEF32F03AEF32F05DC504F15EC5B2
:1064600005F15FC506F160C507F111EC2AF003BF25
:10647000A7EF34F059C13FF55AC140F5B5C541F514
:10648000B6C542F589EC27F036C645F537C646F560
:106490000601406753EF32F0416753EF32F0426735
:1064A00053EF32F0436757EF32F068EF32F00CEC05
:1064B0002BF012EC2BF036C600F137C601F140C6C6
:1064C00004F141C605F111EC2AF003AFA7EF34F057
:1064D0000101036B026B1AC600F11BC601F101AF8B
:1064E00076EF32F0FF0E026FFF0E036F0101076BB4
:1064F000066B1CC604F11DC605F105AF84EF32F032
:10650000FF0E066FFF0E076F16EC2AF00101076BF6
:10651000066B1EC604F11FC605F105AF94EF32F0FD
:10652000FF0E066FFF0E076F16EC2AF00101076BD6
:10653000066B20C604F121C605F105AFA4EF32F0C9
:10654000FF0E066FFF0E076F16EC2AF0D8900101C0
:106550000333023301330033D89001010333023394
:106560000133003300C147F501C148F50101036B58
:10657000026B22C600F123C601F101AFC4EF32F075
:10658000FF0E026FFF0E036F0101076B066B24C63F
:1065900004F125C605F105AFD2EF32F0FF0E066F0C
:1065A000FF0E076F16EC2AF00101076B066B26C67B
:1065B00004F127C605F105AFE2EF32F0FF0E066FDA
:1065C000FF0E076F16EC2AF00101076B066B28C659
:1065D00004F129C605F105AFF2EF32F0FF0E066FA8
:1065E000FF0E076F16EC2AF0D89001010333023337
:1065F00001330033D89001010333023301330033F8
:1066000000C149F501C14AF50101036B026B2AC6BD
:1066100000F12BC601F101AF12EF33F0FF0E026F54
:10662000FF0E036F0101076B066B2CC604F12DC62C
:1066300005F105AF20EF33F0FF0E066FFF0E076F79
:1066400016EC2AF00101076B066B2EC604F12FC66B
:1066500005F105AF30EF33F0FF0E066FFF0E076F49
:1066600016EC2AF00101076B066B30C604F131C647
:1066700005F105AF40EF33F0FF0E066FFF0E076F19
:1066800016EC2AF0D89001010333023301330033B2
:10669000D8900101033302330133003300C14BF5BD
:1066A00001C14CF50101036B026B02C600F103C688
:1066B00001F101AF60EF33F0FF0E026FFF0E036FC9
:1066C0000101076B066B04C604F105C605F105AFB1
:1066D0006EEF33F0FF0E066FFF0E076F16EC2AF019
:1066E0000101076B066B06C604F107C605F105AF8D
:1066F0007EEF33F0FF0E066FFF0E076F16EC2AF0E9
:106700000101076B066B08C604F109C605F105AF68
:106710008EEF33F0FF0E066FFF0E076F16EC2AF0B8
:10672000D89001010333023301330033D8900101C3
:10673000033302330133003300C14DF501C14EF57F
:106740000101036B026B0AC600F10BC601F101AF38
:10675000AEEF33F0FF0E026FFF0E036F0101076B08
:10676000066B0CC604F10DC605F105AFBCEF33F0A6
:10677000FF0E066FFF0E076F16EC2AF00101076B84
:10678000066B0EC604F10FC605F105AFCCEF33F072
:10679000FF0E066FFF0E076F16EC2AF00101076B64
:1067A000066B10C604F111C605F105AFDCEF33F03E
:1067B000FF0E066FFF0E076F16EC2AF0D89001014E
:1067C0000333023301330033D89001010333023322
:1067D0000133003300C14FF501C150F50101036BD6
:1067E000026B12C600F113C601F101AFFCEF33F0EA
:1067F000FF0E026FFF0E036F0101076B066B14C6DD
:1068000004F115C605F105AF0AEF34F0FF0E066F6F
:10681000FF0E076F16EC2AF00101076B066B16C618
:1068200004F117C605F105AF1AEF34F0FF0E066F3D
:10683000FF0E076F16EC2AF00101076B066B18C6F6
:1068400004F119C605F105AF2AEF34F0FF0E066F0B
:10685000FF0E076F16EC2AF0D890010103330233C4
:1068600001330033D8900101033302330133003385
:1068700000C151F501C152F507940501210E326F97
:10688000899A400EC76E200EC66E9E96C69E060E54
:10689000C96EFF0E9EB602D0E82EFCD7898A899A6F
:1068A0009E96C69E020EC96EFF0E9EB602D0E82EC0
:1068B000FCD79E96C69E27C5C9FFFF0E9EB602D086
:1068C000E82EFCD79E96C69E26C5C9FFFF0E9EB633
:1068D00002D0E82EFCD79E96C69E25C5C9FFFF0EA6
:1068E0009EB602D0E82EFCD725EE33F0322F02D030
:1068F00085EF34F09E96C69EDECFC9FFFF0E9EB692
:1069000002D0E82EFCD776EF34F0898A899A9E96D9
:10691000C69E050EC96EFF0E9EB602D0E82EFCD7AD
:106920009E96C69EC952FF0E9EB602D0E82EFCD798
:10693000C9B090EF34F0898A0501200E2527E86A56
:106940002623E86A2723E86A2823FDEC28F01200B2
:1069500021C500F122C501F123C502F124C503F1CF
:10696000899A400EC76E200EC66E9E96C69E0B0E6E
:10697000C96EFF0E9EB602D0E82EFCD79E96C69E2C
:1069800002C1C9FFFF0E9EB602D0E82EFCD79E962C
:10699000C69E01C1C9FFFF0E9EB602D0E82EFCD7ED
:1069A0009E96C69E00C1C9FFFF0E9EB602D0E82E7D
:1069B000FCD79E96C69EC952FF0E9EB602D0E82E08
:1069C000FCD725EE33F00501200E326F9E96C69E51
:1069D000C952FF0E9EB602D0E82EFCD7C9CFDEFF0B
:1069E000322FE6EF34F0898A1200899A400EC76E82
:1069F000200EC66E9E96C69E900EC96EFF0E9EB667
:106A000002D0E82EFCD79E96C69E000EC96EFF0EE1
:106A10009EB602D0E82EFCD79E96C69E000EC96E8A
:106A2000FF0E9EB602D0E82EFCD79E96C69E000EA4
:106A3000C96EFF0E9EB602D0E82EFCD79E96C69E6B
:106A4000C952FF0E9EB602D0E82EFCD7C9CF2DF555
:106A50009E96C69EC952FF0E9EB602D0E82EFCD767
:106A6000C9CF2EF5898A1200FDEC28F0B5C5E8FFE4
:106A7000D70802E3FDEC28F0B5C5E8FFC80802E33B
:106A8000FDEC28F0B5C5E8FFB90802E3FDEC28F0FD
:106A9000B5C5E8FFAA0802E3FDEC28F0B5C5E8FF9C
:106AA0009B0802E3FDEC28F075EC2DF08DEC31F045
:106AB000F29CF29E8B94C69AC290898C9482948C9C
:106AC000720ED36ED3A4FED789968A909390FF0E50
:106AD000E8CF00F0E82EFED7002EFCD78150F294CC
:106AE000F29A9E909D909E929D92F298F292F290D0
:086AF000F286F28E0300FF00A4
:10BF0000E844F926000C160C2B0C3F0C520C640C68
:10BF1000760C860C960CA50CB30CC10CCF0CDC0C6B
:06BF2000E80CF40C000C1B
:00000001FF
